:020000040800F2
:10000000E01E002439030008DB350008772E0008C5
:1000100045030008D5040008C94900080000000095
:10002000000000000000000000000000B33F0008D6
:10003000FB0500080000000071380008B14100080D
:100040005303000853030008530300085303000838
:100050005303000853030008530300085303000828
:100060005303000853030008530300085303000818
:100070005303000853030008530300085303000808
:1000800053030008530300085303000853030008F8
:1000900053030008530300085303000853030008E8
:1000A00053030008530300085303000853030008D8
:1000B00053030008530300085303000853030008C8
:1000C00053030008530300085303000853030008B8
:1000D0005303000885490008530300085303000830
:1000E00053030008530300080000000053030008F6
:1000F0005303000853030008530300085303000888
:100100005303000853030008530300085303000877
:100110005303000853030008530300085303000867
:100120005303000853030008530300085303000857
:100130005303000853030008530300085303000847
:1001400000000000000000000000000000000000AF
:100150005303000853030008530300085303000827
:100160005303000853030008530300085303000817
:100170005303000853030008530300085303000807
:1001800053030008530300085303000853030008F7
:1001900053030008530300085303000853030008E7
:1001A00053030008530300085303000853030008D7
:1001B00053030008530300085303000853030008C7
:1001C00053030008530300085303000853030008B7
:1001D00053030008530300085303000853030008A7
:1001E0005303000853030008530300085303000897
:1001F0005303000853030008530300085303000887
:100200005303000853030008530300085303000876
:100210005303000853030008530300085303000866
:1002200053030008530300085303000800000000B4
:1002300053030008530300080000000053030008A4
:100240005303000853030008530300085303000836
:100250005303000853030008530300085303000826
:100260005303000853030008530300085303000816
:100270005303000853030008530300080000000064
:1002800053030008000000005303000800000000B2
:10029000000000005303000800F002F800F03CF8F2
:1002A0000AA090E8000C82448344AAF10107DA45D1
:1002B00001D100F031F8AFF2090EBAE80F0013F0E7
:1002C000010F18BFFB1A43F001031847E46C00004C
:1002D000046D0000103A24BF78C878C1FAD85207DC
:1002E00024BF30C830C144BF04680C6070470000B0
:1002F0000023002400250026103A28BF78C1FBD82F
:10030000520728BF30C148BF0B6070471FB504F0CB
:10031000EDFC1FBD10B510BD00F0AAF81146FFF7A7
:10032000F5FF04F095FB00F0C8F803B4FFF7F2FF07
:1003300003BC04F05AFB0000094880470948004705
:10034000FEE7FEE7FEE7FEE7FEE7FEE7FEE7FEE785
:10035000FEE7FEE704480549054A064B70470000E2
:10036000B541000899020008E0120024E01E0024B4
:10037000E0140024E0140024704753EA020C00F05B
:1003800069802DE9F04B4FF00006002B1FBFB3FA38
:1003900083F503FA05F424FA05F65E4012BF16430E
:1003A000B2FA82F502FA05F4C5F120051EBF22FA61
:1003B00005FC44EA0C04203556EA044C4FEA144488
:1003C00018BF641C4FF000084FF00009904271EB19
:1003D000030C39D3002919BFB1FA81F701FA07F6E6
:1003E000B0FA80F700FA07F6C7F120071EBF20FA1F
:1003F00007FC46EA0C062037B6FBF4FCA7EB050722
:10040000103F07F01F0BCBF120060CFA0BFB2CFA68
:1004100006F644BFB3460026202FA4BF5E464FF029
:10042000000B5BEA060C08BF4FF0010B19EB0B0940
:10043000ABFB027C48EB0608C01B06FB02CC0BFBA7
:1004400003CC71EB0C01C1E70B460246414648461E
:10045000BDE8F08B13B54FF000004FF00001AFF393
:100460000080BDE81C407047704770477047704778
:10047000754600F02BF8AE4605006946534620F05D
:100480000700854618B020B5FFF764FFBDE820409F
:100490004FF000064FF000074FF000084FF0000B40
:1004A00021F00701AC46ACE8C009ACE8C009ACE8F3
:1004B000C009ACE8C0098D46704710B50446AFF3DB
:1004C00000802046BDE81040FFF72FBF004870476E
:1004D0007C120024FEE70000F0B5BFF34F8FBFF39E
:1004E0006F8F1D4900200860BFF34F8FBFF36F8FE0
:1004F0001A4C216841F400312160BFF34F8FBFF3E4
:100500006F8F164970310860BFF34F8F081F006866
:1005100043F6FF75104E1036C0F34E31C0F3C903D9
:1005200005EA4112184642EA80773760401EFAD247
:10053000491EF5D2BFF34F8F206840F48030206011
:10054000BFF34F8FBFF36F8F03484C30016841F00A
:1005500004010160F0BD000050EF00E014ED00E088
:100560002DE9F0430D4F00241D461646884681466E
:1005700004EB041017F81010B14209D107EB400149
:100580004878A84204D1891C4246484600F02AF81F
:10059000641CA4B2382CEBD3BDE8F083F6640008E9
:1005A0002DE9F0430E4F00241D461646884681462D
:1005B00004EB840000EB441017F81010B14209D18D
:1005C00007EB40014878A84204D1891C42464846BE
:1005D00000F008F8641CA4B2092CE9D3BDE8F0834C
:1005E000CC6C0008002310B504E011F8014B5B1C33
:1005F00000F8014B9342F8D310BD7047F0B51C468C
:10060000094B0A4F164685B04FF0000C10251A888A
:100610005B883F88121A5B1A8DE8F01092B29BB289
:1006200000F0A4F905B0F0BD6C1200242C000024E9
:100630002DE9FF411C46084B1646002710251A8855
:100640005B88121A5B1A8DE8F00092B29BB203F03D
:10065000FDFCBDE8FF8100006C1200242DE9F04193
:100660001546DFF85C8001220C460646404617031B
:10067000394600F05EFB052000F0D6F9032003F0B8
:10068000E1FBC4F3074003F0DDFBC4F3072003F0F4
:10069000D9FBE0B203F0D6FB002405E0FF2003F015
:1006A000D1FB3055641CA4B2AC42F7D300223946CA
:1006B000404600F03EFBBDE8F041052000F0B4B933
:1006C0000004025830B40C460178202A1AD009DC04
:1006D0000C2A0DD0102A13D0182A17D10C4801FB70
:1006E000030108E0302A0FD0402A0FD10948F6E76D
:1006F000594301F50021204630BC1A46FFF7AEBF32
:100700000548ECE70548EAE70548E8E730BC7047EC
:1007100000120800009208000008080000260800E7
:100720000048080030B40C460146007815464A7867
:10073000812809D3402A07D3FF2A05D0FF2803D0F8
:100740007F2A0CD2403A0BE00022104603E0521CF4
:1007500092B204F8010B9A42F9D330BC7047413A87
:100760008138C0B2D1B2C0EB401202EB801001EB75
:10077000400159430C2D0CD0102D0CD0182D0DD04C
:10078000202DEAD101F56011204630BC1A46FFF752
:1007900065BF044800E004480144F5E701F5ED11A8
:1007A000F2E700000014090000DD1100AFF3008043
:1007B00070B586B04FF6FF7002F0D0FB00206C469B
:1007C00005462554401CC0B21828FAD311222046F1
:1007D0000021FFF743FF10216B464FF4784608468F
:1007E0003246FFF70BFF00202554401CC0B21828EA
:1007F000FAD3082268461421FFF730FF20216B4608
:1008000010203246FFF7FAFE00202554401CC0B2EB
:100810001828FAD3082268461E21FFF71FFF30214F
:100820006B4610203246FFF7E9FE4FF4FA6004F001
:10083000E7F806B070BD2DE9F04FC1B01C46164672
:100840000D4682468946580701D0012100E000216B
:1008500001EBD40061080C2C10FB01F0834609D099
:10086000102C07D0182C05D0202C03D0302C01D010
:10087000402C2DD10346224669463046FFF722FF21
:10088000002022E01DF808700026380601D54A9A9B
:1008900002E04C9820B94B9A2946504602F0C0FB22
:1008A00078066D1CADB2070EA5EB0900A04205D17C
:1008B0000AF101004D461FFA80FA03E0761CB6B239
:1008C000082EE2D308F1010080B258458046D9D302
:1008D00041B0BDE8F08F2DE9F04FA1B01F4615469D
:1008E0000C4682468946580701D0012100E00021CC
:1008F00001EBD7000C2F10FB07F0834605D0102F1B
:1009000003D0182F01D0202F2DD103463A46694637
:100910002846FFF707FF002022E01DF808600025A9
:10092000300601D52A9A02E02C9820B92B9A21464C
:10093000504602F075FB7006641CA4B2060EA4EBD0
:100940000900B84205D10AF101004C461FFA80FAAD
:1009500003E06D1CEDB2082DE2D308F10100C0B236
:1009600058458046D9D321B0BDE8F08F2DE9FF4F1F
:1009700083B09B460E46044680468A46DDE91075E4
:100980000020814620E0B9F1000F23D005994FF0F7
:10099000000908EB0100401BA04202DA701944462E
:1009A00086B20AEB0B00401BB04210DB12AB93E89F
:1009B00007002B468DE807003A4631462046FFF7F0
:1009C0008AFF601984B2BF1C38780028DBD107B0D9
:1009D000BDE8F08F802801D90120D2E7059A08EB05
:1009E0000201A1EB5501A14202DA711944468EB20F
:1009F0000AEB0B01491BB142E9DB0D280FD012AB0A
:100A000093E807002B468DE807003A46314620461A
:100A1000FFF711FF04EB550084B27F1CD4E7701977
:100A2000444686B27F1CF5E7002206E00021491CFF
:100A3000C9B26429FBD3521CD2B28242F6D37047AA
:100A400070B4164602781D464378812A0C4610D3AE
:100A5000402B0ED3FF2B0CD0FF2A0AD00C2D11D027
:100A6000102D11D0182D0DD13146204670BCFFF746
:100A700097BD0021084603E0491C04F8010BC9B2E8
:100A8000B142F9D370BC70473146204670BCFFF7C5
:100A900067BD000010B528B190F83510022903D0C9
:100AA00080214165012010BD1D4A4FF49563016806
:100AB0008C189C4207D8042280F83520086820F062
:100AC0000100086029E00C6824F00E040C60016845
:100AD0000A440A6822F001020A60016E0A6822F4E0
:100AE00080720A6090F85C30012202FA03F10D4B2B
:100AF0001960D0E919134B60C16E31B10B6823F452
:100B000080730B60D0E91C134B60002180F8341017
:100B100080F83520016D01B18847002010BD00002C
:100B2000F0FFFDBF045402580248016841F0010182
:100B300001607047200400582DE9F84F6C4C0022EA
:100B40004FF0B04A4FF0010B4FF0030E4FF00F097A
:100B50000B680BFA02F73B40BB4270D14D68022D87
:100B600001D0122D12D1D50800EB850CDCF82060E5
:100B70005507ED0E09FA05F826EA0806D1F81080A7
:100B800008FA05F848EA0608CCF82080D0F800807A
:100B9000560091F804C00EFA06F50CF0030C28EA92
:100BA00005080CFA06FC4CEA080CC0F800C0D1F8A5
:100BB00004C0BCF1010F08D0BCF1020F05D0BCF19C
:100BC000110F02D0BCF1120F16D1D0F808C0D1F825
:100BD0000C802CEA050C08FA06F848EA0C08C0F864
:100BE0000880D0F804C02CEA070C0F79C7F300176F
:100BF000974047EA0C074760C768AF438D68B54028
:100C00003D43C5604D68ED006BD53A4D2E6846F00A
:100C100002062E602D6822F0030606F1B04605F0AC
:100C200002050095D6F808C495072F0F09FA07F5B5
:100C30002CEA050C304DA84202D100252EE050E0F0
:100C40002E4DA84201D1012528E02D4DA84201D109
:100C5000022523E02B4DA84201D103251EE02A4D99
:100C6000A84201D1042519E0284DA84201D105254B
:100C700014E0274DA84201D106250FE0254DA842DA
:100C800001D107250AE0244DA84201D1082505E03D
:100C9000224DA84201D1092500E00A25BD4045EAC0
:100CA0000C05C6F8085425684E689D43F60300D528
:100CB0001D43256065684E689D43B60300D51D43FE
:100CC0006560DAF8005056464F689D43FF0200D534
:100CD0001D43356075684F689D43BF0200D51D43B5
:100CE0007560521C102AFFF433AFBDE8F88F000086
:100CF00080000058F44402580000025800040258D2
:100D000000080258000C0258001002580014025843
:100D100000180258001C02580020025800240258F3
:100D20000069084000D00120704742694A40426192
:100D300070470AB10183704741837047014880685A
:100D400070470000180000240248816802781144AE
:100D50008160704718000024032010B500F0A2F84D
:100D60000F2000F007F808B1012010BD00F06CF86A
:100D7000002010BD70B50D4D04464FF47A712878EF
:100D8000B1FBF0F00A490968B1FBF0F001F0A0FEF8
:100D900048B9102C07D200222146501E00F062F8FC
:100DA00000206C6070BD012070BD000018000024A0
:100DB00008000024134A41781160111D03780A1DB0
:100DC000E3B143680B60017BC37A090741EA036121
:100DD000837A41EAC341437B41EA8341837B41EA11
:100DE0004341C37B41EA0341437A41EA0321037A49
:100DF000007841EA43010143116070470020086018
:100E00001060704798ED00E0BFF35F8F0448016801
:100E100021F4803101600249002070310860704780
:100E200024ED00E0074940F00100086005487038F3
:100E3000016841F480310160BFF34F8FBFF36F8FC2
:100E40007047000094ED00E07047002809DB0121A5
:100E500000F01F0291404009800000F1E020C0F83E
:100E6000001170470E4BF0B41B68C3F30223C3F1AB
:100E70000704042C00D904241D1D072D01D20023D2
:100E800000E0DB1E012606FA04F56D1E0D409D40B4
:100E90009E40761E164045EA0601F0BC03F095BD63
:100EA0000CED00E0064A00F0070110684FF6FF0362
:100EB000184040EA012003490843106070470000D1
:100EC0000CED00E00000FA052DE9F84F17468B46BF
:100ED0000446FFF733FF824694F8400001280ED005
:100EE000012684F8406094F841004FF00008012882
:100EF00007D0022584F840802846BDE8F88F0220FC
:100F0000FBE7C4F844804FF0020984F841900022C6
:100F1000202153462046009702F052FE0500E9D1F9
:100F200000225946204602F0A4FCDBF8240058B900
:100F30000122534602212046009702F041FE05009F
:100F4000D8D12168C1F80C9084F84160D2E7000044
:100F5000F8B50446FFF7F2FE07465CB194F840008E
:100F6000012809D0012684F8406094F8410000254A
:100F700020B10BE00120F8BD0220F8BD84F84050FC
:100F8000204600F051F841F28830A06420680168E2
:100F90004FF4706393FAA3F321F47062A168B3FA7B
:100FA00083F3491E99400A430260A06C002220216D
:100FB0003B460090204602F003FE70BB4FF07F4797
:100FC000E268E16997FAA7F763680A43216AB7FA0A
:100FD00087F7BB4019430A4321680B68104F3B4019
:100FE0001A430A60D4E905310B4321684A684FF47B
:100FF000F81C0C4F9CFAACFC3A402769BCFA8CFCFC
:1010000007FA0CF73A4313434B6021680A6842F031
:1010100001020A60656484F8416084F84050F8BDBC
:101020002FFFFF00FEF8E0FF2D482DE9F043016897
:1010300087B041F480410160006800F48040059071
:1010400027480C30016841F002010160016801F09D
:1010500002010591016841F008010160016801F099
:1010600008010591016841F0100101600068022447
:101070000325DFF8709000F01000059040206946CD
:10108000CDE900040120CDE902050A20049048467C
:10109000FFF752FD00264FF004080927CDF8008025
:1010A00069464846CDE90146CDE90357FFF744FDBF
:1010B0004FF4605069468DE851000B48CDE9035765
:1010C000FFF73AFDCDF800806946CDE901460748B3
:1010D000CDE90357FFF730FD07B0BDE8F08300000E
:1010E000D444025800040258000C02580010025860
:1010F0002DE9F84F16460F460446FFF71FFE8246BD
:101100002068816900F1200594F84020012A0ED062
:101110004FF0010884F8408094F841204FF0000916
:10112000012A06D0022084F84090BDE8F88F022002
:10113000FBE7C4F8449097B3222284F84120026967
:10114000521CA2630269521C62632763426922F047
:10115000406242F080624261206881610CE00621B9
:10116000204602F02DFDB8B92A78206B411C21637E
:101170000270A06B401EA063A06B53464FF00102AB
:1011800000960028EBD14FF00201204602F018FD36
:1011900010B922680221D16084F84180C3E7FFE7DB
:1011A000606C40F0080060640120BCE72DE9F84F56
:1011B00016460F460446FFF7C1FD8246206894F8A4
:1011C000401000F1200501290ED04FF0010884F8ED
:1011D000408094F841104FF00009012906D0022008
:1011E00084F84090BDE8F88F0220FBE7C4F84490F3
:1011F00077B3122184F841100169491CE162016949
:10120000491CA1626762416921F0406141610CE0C3
:101210000421204602F0D4FCB8B9606A411C616226
:1012200000782870E06A401EE062E06A53464FF0A2
:10123000010200960028EBD14FF00201204602F097
:10124000BFFC10B922680221D16084F84180C7E751
:10125000606C40F0080060640120C1E710B500F048
:10126000B3FE084909684FF4807292FAA2F201F4C1
:101270007061B2FA82F2D140034A515CC84003491E
:10128000086010BD184402580E4D000808000024E4
:1012900010B500F053FE07490968102292FAA2F235
:1012A00001F07001B2FA82F2D140034A515CC840A9
:1012B00010BD0000204402580E4D0008364930B5DC
:1012C0000A68096812F00302344BC1F305311B6848
:1012D000334C03F010032468DFED320AB7EE001A36
:1012E000C4F3CC0414FB03F300EE103A2E4BB8EE1B
:1012F000400A07D02D4C012A01D0022A4AD0B4FB63
:10130000F1F10BE0244C283C22689506284A03D5CD
:101310002468C4F3C104E240B2FBF1F101EE901A7B
:101320001968B8EE612AC1F3080101EE901A196834
:10133000F8EE611A40EE201A31EE810A22EE000A20
:10134000C1F34621491C00EE901AF8EE600A80EEC7
:10135000201AFCEEC10AC0ED000A1968C1F306416B
:10136000491C00EE901AF8EE600A80EE201AFCEE9E
:10137000C10AC0ED010A1968C1F30661491C00EEFB
:10138000901AF8EE600A80EE201ABCEEC10A80EDD9
:10139000020A30BD074ABFE7284402582C440258CD
:1013A0003C440258000000393844025800093D000E
:1013B0000090D00340787D01364930B50A6809684D
:1013C00012F00302344BC1F305511B68334C03F494
:1013D00080732468DFED320AB7EE001AC4F3CC0440
:1013E00014FB03F300EE103A2E4BB8EE400A07D080
:1013F0002D4C012A01D0022A4AD0B4FBF1F10BE0B6
:10140000244C283C22689506284A03D52468C4F356
:10141000C104E240B2FBF1F101EE901A1968B8EE96
:10142000612AC1F3080101EE901A1968F8EE611AF9
:1014300040EE201A31EE810A22EE000AC1F3462165
:10144000491C00EE901AF8EE600A80EE201AFCEEBD
:10145000C10AC0ED000A1968C1F30641491C00EE3B
:10146000901AF8EE600A80EE201AFCEEC10AC0ED78
:10147000010A1968C1F30661491C00EE901AF8EEE2
:10148000600A80EE201ABCEEC10A80ED020A30BD6F
:10149000074ABFE7284402582C44025844440258E3
:1014A000000000394044025800093D000090D0037C
:1014B00040787D012DE9F84F0446006800252E464E
:1014C000010104F12400FE4FDFF8F88300901DD5E0
:1014D000606E50B1B0F5801F0CD0B0F5001F0ED07B
:1014E000B0F5401F1DD001250FE0386840F40030F2
:1014F000386016E00221201D02F086FB03E0009810
:10150000022102F0F9FB05000BD02E462088C00511
:1015100023D5606D05281ED2DFE800F00C11161BE4
:101520001B00D8F80010626E21F440111143C8F876
:101530000010EBE7386840F40030386009E0002123
:10154000201D02F061FB03E00098002102F0D4FBB3
:1015500005466DB100E001252E432088800528D581
:10156000A06D80281ED00CDC90B140280ED114E074
:10157000D8F80010626D21F007011143C8F800107F
:10158000EBE7C02813D0B0F5807F10D001250FE025
:10159000386840F40030386009E00021201D02F076
:1015A00033FB03E00098002102F0A6FB054685B15D
:1015B0002E432088DFF8109340052CD5D4F8A400E2
:1015C000B0F5800F20D00DDCA0B1B0F5001F0FD119
:1015D00015E0D8F80010A26D21F4E0711143C8F8AD
:1015E0000010E6E7B0F5C00F13D0B0F5000F10D033
:1015F00001250FE0386840F40030386009E0002130
:10160000201D02F001FB03E00098002102F074FBB2
:10161000054675B12E43208800052DD5D4F8A800C5
:10162000B0F1007F21D00EDCA8B1B0F1807F10D1E5
:1016300016E0D9F80010D4F8A42021F46001114379
:10164000C9F80010E7E7B0F1407F13D0B0F1806F28
:1016500010D001250FE0386840F40030386009E010
:101660000021201D02F0D0FA03E00098002102F0D2
:1016700043FB05466DB12E43206880011FD5A06C49
:10168000D8B110280FD0202812D0302815D001252D
:1016900014E0D9F80010D4F8A82021F0E06111433B
:1016A000C9F80010E8E7386840F40030386004E01A
:1016B0000221201D02F0A8FA05466DB12E432088B4
:1016C000C0042BD5E06DB0F5005F20D00DDCA0B1DB
:1016D000B0F5805F0FD115E07A48001F0168A26C59
:1016E00021F0300111430160E9E7B0F5405F13D00C
:1016F000B0F5804F10D001250FE0386840F400307D
:10170000386009E00021201D02F07EFA03E0009815
:10171000002102F0F1FA054685B12E4320888004AD
:1017200029D5206EB0F5403F23D010DC08B3B0F5CA
:10173000803F14D0B0F5003F0FD115E0D8F800106D
:10174000E26D21F4E0411143C8F80010E6E7B0F57E
:10175000802F0ED0B0F5A02F0BD001250AE001217B
:10176000201D02F051FA03E00098012102F0C4FAB2
:1017700005468DB12E43208840042AD5D4F8AC000C
:10178000B0F1405F23D010DC08B3B0F1805F14D01B
:10179000B0F1005F0FD115E0D8F80010226E21F4EF
:1017A000E0211143C8F80010E5E7B0F1804F0ED0FA
:1017B000B0F1A04F0BD001250AE00121201D02F05D
:1017C00023FA03E00098012102F096FA05466DB174
:1017D0002E43208800041FD5E06ED8B1B0F1805FA1
:1017E0000ED0B0F1005F10D0012514E0D9F8001040
:1017F000D4F8AC2021F0E0411143C9F80010E8E72B
:10180000386840F40030386004E00121201D02F007
:10181000FBF905466DB12E432068C0011ED5606CF2
:10182000D0B101280ED0022811D0032814D00125F0
:1018300013E0D8F80010E26E21F040511143C8F8CF
:101840000010E9E7386840F40030386004E0022115
:10185000201D02F0D9F9054675B12E432068DFF846
:101860006CB040025AD51A48016841F48071016099
:10187000FFF764FA82460EE01248001F0168626CAE
:1018800021F0030111430160E8E7FFF757FAA0EBED
:101890000A0064283AD80E480068C005F5D5B5BBE3
:1018A000094818300068B4F8B01000F4407001F432
:1018B0004071884219D00448183001680AE00000DD
:1018C0002C440258504402585844025810440258BC
:1018D00000480258026821F4407142F480320260EC
:1018E000026822F4803202600160D4F8B000B0F5E2
:1018F000807F22D1FFF722FA824609E0FFF71EFA25
:10190000A0EB0A0141F28830814201D9032504E0AD
:10191000FE4800688007F1D57DB12E432078DFF8BE
:10192000F0A3C0073CD0A06F182837D025DC78B3CF
:10193000082828D0102824D12BE0D4F8B000C0F318
:10194000012103290ED0DBF8001021F47C51CBF8E3
:101950000010EE480168B4F8B020C2F30B02114346
:101960000160DBE7DBF80020EA4B22F47C5203EA5B
:1019700010100243CBF80020EBE720280ED02828D7
:101980000CD001250BE00121201D02F03DF904E0FF
:1019900004E00098012102F0AFF905465DB12E4345
:1019A000207880071ED5606F062819D2DFE800F086
:1019B000160C11161616DAF80010A26F21F0380175
:1019C0001143CAF80010EBE70121201D02F01CF9B9
:1019D00003E00098012102F08FF9054675B100E09F
:1019E00001252E43207840071FD5D4F89000062803
:1019F00019D2DFE800F0160C11161616DAF80010EE
:101A0000626F21F007011143CAF80010EAE70121D3
:101A1000201D02F0F9F803E00098012102F06CF9B2
:101A200005469DB100E001252E43207880062BD588
:101A3000D4F88C00B0F1405F24D011DC10B3B0F1C9
:101A4000805F15D0B0F1005F10D116E0D9F800101A
:101A5000D4F8902021F007011143C9F80010E4E701
:101A6000B0F1804F0ED0B0F1A04F0BD001250AE0AD
:101A70000021201D02F0C8F803E00098022102F0C6
:101A80003BF905468DB12E43207840062BD5D4F87E
:101A90009800B0F5406F24D011DC10B3B0F5806F22
:101AA00015D0B0F5006F10D116E0DAF80010D4F8B8
:101AB0008C2021F0E0411143CAF80010E4E7B0F5B2
:101AC000805F0ED0B0F5A05F0BD001250AE00021A9
:101AD000201D02F099F803E00098022102F00CF9B1
:101AE00005468DB12E43207800062BD5D4F89C00F6
:101AF000B0F5C04F24D011DC10B3B0F5005F15D0A5
:101B0000B0F5804F10D116E0D9F80010D4F8982025
:101B100021F4E0511143C9F80010E4E7B0F5004F9B
:101B20000ED0B0F5204F0BD001250AE00021201D7A
:101B300002F06AF803E00098022102F0DDF80546A1
:101B400065B32E43207800070BD5D4F88000B0F59C
:101B5000805F2DD0DAF8002022F440520243CAF808
:101B600000202078C0060BD5D4F89400B0F5807F13
:101B700024D0D9F8002022F440720243C9F8002092
:101B8000206800032CD5D4F8A000E8B1B0F5803F60
:101B90001FD0B0F5003F21D0012520E0D9F800107A
:101BA000D4F89C2021F460411143C9F80010C9E722
:101BB0000098022102F0A0F80643D2E70098022123
:101BC00002F09AF80643DBE70021201D02F01CF822
:101BD00003E00098022102F08FF8054685B12E43FC
:101BE0002068400322D5D4F88400B0F5801F11D0BE
:101BF000B0F5001F13D0B0F5401F15D0012514E03B
:101C0000D9F80010D4F8A02021F440311143C9F8CC
:101C10000010E5E7386840F40030386004E00098D0
:101C2000012102F069F8054655B12E432068C00332
:101C30001CD5E06C70B1B0F5803F10D0012514E0E8
:101C4000DAF80010D4F8842021F440111143CAF8C6
:101C50000010EBE7386840F40030386004E00221FF
:101C6000201D01F0D1FF0546C5B12E43206880003C
:101C700004D50098022102F03FF806432068800353
:101C80001BD5E06FB8B1B0F5807F10D0B0F5007F04
:101C900011D0B0F5407F0ED001250DE01C4808386A
:101CA0000168E26C21F4803111430160DEE738689D
:101CB00040F40030386045B32E432068C00207D599
:101CC000D8F80000226F20F000401043C8F8000050
:101CD0002068C00008D5DBF80010D4F8B42021F447
:101CE00080411143CBF800102068800207D5D8F856
:101CF0000010A26E21F080711143C8F80010206816
:101D0000400014D5DBF8001006E01EE070440258D5
:101D100054440258CFFFFF0021F40041CBF80010DB
:101D2000DBF80010D4F8B8201143CBF8001020687D
:101D3000002806DA0A480168226D21F0405111435B
:101D400001605EB10120BDE8F88FDAF80010E26FA3
:101D500021F440711143CAF80010AEE70020F2E709
:101D60004C4402582DE9F047DFF8BC9104460E467A
:101D7000D9F8000000F00700B0420CD2D9F80010EA
:101D800021F007013143C9F80010D9F8000000F034
:101D90000700B0427ED12078DFF89081800707D518
:101DA000D8F80010E26821F00F011143C8F80010C4
:101DB0002078C00762D0D8F80010A26821F47061C2
:101DC0001143C8F8001059496068183902281CD01E
:101DD00003281DD0096801281DD04907002960DAB1
:101DE000524F083F396821F0070101433960FEF77F
:101DF000A5FF0546606841F28831022813D0032808
:101E00001ED001288A4627D034E009688903E5E717
:101E100009688901E2E7C905E0E7FEF78FFF411B8A
:101E2000514501D923E08A463868C0F3C200022830
:101E3000F3D123E0FEF782FF411B514501D916E0A3
:101E40008A463868C0F3C2000328F3D116E0FEF7D3
:101E500075FF411B51450AD83868C0F3C2000128FC
:101E6000F5D10BE0FEF76AFF411B514502D9032073
:101E7000BDE8F087386810F0380FF3D1D9F80010BA
:101E8000484601F00701B1420DD9016821F0070170
:101E9000314300E005E00160006800F00700B04257
:101EA00001D00120E4E72078400707D5D8F80010DA
:101EB000226921F070011143C8F800102078010751
:101EC0001B4805D50168626921F07001114301606A
:101ED0002178C90605D50168A26921F4E0611143A2
:101EE00001602078800607D51149091D0868E2695C
:101EF00020F070001043086000F066F8D8F8001079
:101F00004FF4807292FAA2F201F47061B2FA82F296
:101F1000D140084A515CC840074908600F20FEF7CD
:101F200029FF0020A4E700000020005218440258B6
:101F30001C4402580E4D00080800002410B5FFF79D
:101F40008DF908490968012292FAA2F201F00F0105
:101F5000B2FA82F2D140044A515CC8400349086099
:101F600010BD0000184402580E4D00080C0000245B
:101F700010B5FFF7E3FF07490968102292FAA2F2B1
:101F800001F07001B2FA82F2D140034A515CC840BC
:101F900010BD00001C4402580E4D000810B5FFF79C
:101FA000CDFF074909684FF4807292FAA2F201F45A
:101FB000E061B2FA82F2D140024A515CC84010BDE1
:101FC0001C4402580E4D00083548F0B50068364DE7
:101FD00010F03801334809D00411082904D0334ED9
:101FE00010290BD018290BD02046F0BD296889068E
:101FF000FBD52968C1F3C101C840F0BD3046F0BD32
:10200000274918310A68096812F00302284BC1F306
:1020100005111B68274F03F001033F68DFED260A17
:10202000B7EE001AC7F3CC0717FB03F300EE103A24
:10203000224BB8EE400A06D0012A01D0022A2BD04A
:10204000B4FBF1F008E02A68920603D52A68C2F3CF
:10205000C102D040B0FBF1F001EE900A1868B8EE72
:10206000612AC0F3080001EE900A1868F8EE611AC0
:1020700040EE201A31EE810A22EE000AC0F346201B
:10208000401C00EE900AF8EE600A80EE201ABCEECA
:10209000C10A10EE100AF0BDB6FBF1F0DCE700005B
:1020A000104402580090D0030044025840787D014B
:1020B0002C4402583444025800000039304402587D
:1020C0002DE9F05F04460078DFF8FC8341F288399F
:1020D000DFF8F8A3FE4DC0074ED0D8F800104046F8
:1020E000C1F3C20102291AD00068C0F3C20003285C
:1020F00005D1DAF8000000F0030002280FD0606874
:10210000B0F5803F12D010B1B0F5A02F19D02868DB
:1021100020F480302860286820F4802009E02868B6
:10212000800329D56068002874D025E0286840F431
:1021300080302860606890B1FEF700FE06464F468A
:1021400009E0286840F480202860EFE7FEF7F6FDFC
:10215000801BB8427DD828688003F7D50CE0FEF7D5
:10216000EDFD06464F4604E0FEF7E8FD801BB84251
:10217000F0D828688003F7D42078D64F80075AD546
:10218000D8F8001040464FF47C3B11F0380F13D0C4
:102190000068C0F3C200032803D1DAF8000080070A
:1021A0000AD0E068A8B3296821F019010143296029
:1021B000FEF7C4FD06461DE02868400702D5E0682A
:1021C0000028B1D02868E16820F019000843286091
:1021D000FEF7B4FD064604E0FEF7B0FD801B0228C2
:1021E000B8D828684007F7D507E0FEF7A7FD801BA1
:1021F0000228AFD828684007F7D538689BFAABF2B9
:1022000020F47C312069B2FA82F2904001433960B7
:1022100011E000E0AEE0286820F001002860FEF741
:102220008DFD064604E0FEF789FD801B022891D84B
:1022300028684007F7D42078C00655D5D8F8001094
:1022400040464FF0F84BC1F3C201012917D0006896
:1022500000E0EDE0C0F3C200032805D1DAF8000089
:1022600000F0030001280AD0E069002828682CD07B
:1022700040F080002860FEF761FD064616E0286801
:10228000C00502D5E069802874D138689BFAABF2AA
:1022900020F0F841206AB2FA82F29040014339609E
:1022A00022E0FEF74BFD801B022899D82868C00564
:1022B000F7D538689BFAABF2216AB2FA82F220F0C5
:1022C000F8409140084338600EE020F0800028601C
:1022D000FEF734FD064604E0FEF730FD801B0228C1
:1022E00087D82868C005F7D42078000724D5774F11
:1022F00060694C37002838680FD040F00100386022
:10230000FEF71CFD064604E0FEF718FD801B0228C0
:102310008DD838688007F7D50EE020F001003860CE
:10232000FEF70CFD064604E0FEF708FD801B0228C0
:102330007ED838688007F7D42078800623D5A06936
:10234000002828680FD040F480502860FEF7F6FC83
:10235000064604E0FEF7F2FC801B022868D82868D5
:102360008004F7D50FE020F480502860FEF7E6FCEB
:10237000064605E0D6E0FEF7E1FC801B022857D8B0
:1023800028688004F7D42078400744D5524F386835
:1023900040F480703860FEF7D1FC064604E0FEF79A
:1023A000CDFC801B642843D83868C005F7D5474F5B
:1023B000A068483701280AD008B1052811D038682C
:1023C00020F001003860386820F0040002E038682E
:1023D00040F001003860A06888B1FEF7AFFC064607
:1023E00009E0386840F004003860F0E7FEF7A6FC2A
:1023F000811B49451CD838688007F7D50BE0FEF7EC
:102400009DFC064604E0FEF799FC811B49450FD868
:1024100038688007F7D4606AF0B3D8F80010C1F3C9
:10242000C20103297ED00228286820F0807000E0D5
:1024300079E0286003D0FEF781FC044687E0FEF7D0
:102440007DFC064604E0FEF779FC801B02287BD861
:1024500028688001F7D4DAF8001040F2F332914393
:10246000E26A41EA0211A26A1143CAF8001094F824
:1024700034004FF4FE02218E4002491EA0F5007088
:1024800080B2C1F308010843218F491E02EA0141CD
:10249000084394F83C1000E05CE0491E120202EA96
:1024A000016108430949083108600B1D19684FF69E
:1024B000F872A06C914392FAA2F2B2FA82F29040C2
:1024C00001431960014809E01044025828440258A9
:1024D000004402580444025800480258001D016894
:1024E000226C21F00C01114301600168626C21F043
:1024F000020111430160016841F48031016001680B
:1025000041F400310160016841F4802101600168FB
:1025100041F001010160286840F080702860FEF7FA
:102520000DFC01E018E00FE0044604E0FEF706FCB5
:10253000001B022808D828688001F7D50AE0FEF7BA
:10254000FDFB001B022802D90320BDE8F09F28688C
:102550008001F4D40020F8E70120F6E72DE9F05FD0
:1025600004004FF000053DD0DFF8C4812068714EB3
:10257000714F4045A36A06D0B04204D0B84202D0A1
:10258000E1680F292ED8E26B4FF0010B0BEB521CC8
:10259000E26802F10801C908404501FB0CF105D0D1
:1025A000B04203D0B84201D008291BD8404503D01F
:1025B000B04201D0B84201D1102913D84FF480099C
:1025C0004B4512D1404507D0B04205D0B84203D0A8
:1025D000206BB0F5702F05D8256B05B91504B2EB4B
:1025E000154F02D90120BDE8F09F94F881004FF00B
:1025F000000A20B9204684F880A000F09FF802204D
:1026000084F881002068016821F001010160A0695F
:10261000B0F1806F09D16068484506D1A06B20B940
:102620002068016841F480510160A16AE0690843B3
:10263000E16B29430843E168084321688860616AC7
:10264000606BA2690843A16B1143084321690843E9
:1026500061690843216A084361680843E16C0843E3
:10266000A1680843A16C0843A16D08432168C860B4
:10267000A06A484529D1206C01282068016827D02C
:1026800021F400410160606C01282068016822D0BB
:1026900021F4804101602068404506D0B04204D05A
:1026A000B84202D0B5F5702F18D0404503D0B042E3
:1026B00001D0B84202D1B5F5F81F0FD0016821F45E
:1026C000005101602168E06A0864606850B119E057
:1026D00041F40041D6E741F48041DBE7016841F471
:1026E0000051EEE7A06A30B92068816821F4C0513A
:1026F00041F4006181602068816821F4C06141F487
:10270000806181602068016D21F0010101656068D0
:10271000400206D52068C168626D21F00041114376
:10272000C160C4F884A084F881B000205BE7000099
:102730000030014000380040003C0040164800B521
:10274000B5B0016841F002010160006800F00200CC
:10275000349011480830016841F4804101600068FC
:1027600000F4804034904FF4805000900020179087
:102770006846FEF79FFE4FF460402F900220309095
:1027800001203190032032900520339003482FA977
:10279000FEF7D2F935B000BDE044025800040258FB
:1027A0002DE9F84F044690F880001F4692460A9D96
:1027B00001288B4613D04FF0010984F88090FEF772
:1027C000BDFA94F8812006460020012A4FF48001CA
:1027D0000ED062688A4209D1A2683AB902E00220AA
:1027E000BDE8F88F94F88120042A01D0022136E058
:1027F000BBF1000F32D0BAF1000F2FD077B394F8AD
:102800008120042A02D0052284F881208046C4F861
:102810008400C4F864A0A4F86A70A4F86870C4F8CE
:102820005CB0A4F86270A4F86070206760672068EC
:1028300042686FF30F023A4342602068026842F038
:10284000010202606068884204D12068016841F496
:1028500000710160E0680F2840D848E0012184F849
:1028600080000846BCE7B4F8620070B12068416996
:1028700089070AD5E16D09680162E06D001DE06518
:10288000B4F86200401EA4F86200B4F86A0080B197
:102890002068416948F2080211420AD0006B616E5B
:1028A0000860606E001D6066B4F86A00401EA4F8FF
:1028B0006A00681C12D0FEF741FA801BA8420DD3B3
:1028C000204601F0E7FA84F88080D4F8840040F4D0
:1028D0008070C4F8840084F88190EBE0B4F8620062
:1028E0000028C0D1B4F86A000028BCD1C8E007288D
:1028F00049D8BDE0B4F86200F0B1206841698907A9
:102900001AD5B4F8621001290BD9E16B49B1E16D18
:1029100009680162E06D001DE065B4F86200801E88
:1029200008E0E16D09880184E06D801CE065B4F881
:102930006200401EA4F86200B4F86A00E0B12068AA
:10294000416911F4604F17D04169090409D5006B42
:10295000616E0860606E001D6066B4F86A00801EDB
:1029600008E0008E616E0880606E801C6066B4F8BE
:102970006A00401EA4F86A00681C04D0FEF7DEF965
:10298000801BA8429CD2B4F862000028B2D1B4F8EF
:102990006A000028AED173E0B4F8620080B320680A
:1029A000416989072CD5B4F8621003290CD9E16B71
:1029B000402909D9E16D09680162E06D001DE065FB
:1029C000B4F86200001F19E0B4F8621001290BD9B5
:1029D000E16B49B1E16D09880184E06D801CE0651F
:1029E000B4F86200801E09E0E16D097880F82010DB
:1029F000E06D401CE065B4F86200401EA4F862007F
:102A0000B4F86A0068B32068416911F4604F28D0B7
:102A10004169090409D5006B616E0860606E001D94
:102A20006066B4F86A00001F19E0416901F4C04112
:102A3000B1F5005F09D9008E616E0880606E801C60
:102A40006066B4F86A00801E09E090F83000616E9C
:102A50000870606E401C6066B4F86A00401EA4F8FE
:102A60006A00681C04D0FEF769F9801BA84289D26D
:102A7000B4F8620000288FD1B4F86A0000288BD126
:102A80000022334608212046009501F072FA28B151
:102A9000D4F8840040F02000C4F88400204601F0FF
:102AA000F9F984F8808084F88190D4F884000028B3
:102AB0003FF4D8AE012093E64FF0E02104280869E6
:102AC00003D020F004000861704740F00400FAE7EA
:102AD000401EB0F1807F10B501D3012010BD4FF032
:102AE000E02460610F21601701F06FFF0020A061FA
:102AF00007202061002010BD7047704790F87910C2
:102B000090F87A000843704770B502680446D069AF
:102B10001368916810F00F0F64D0594D03F490764C
:102B20000D40354376D0C50707D0DD0505D5012515
:102B30001562E26F42F00102E267820708D5CA0718
:102B400006D0256802222A62E26F42F00402E267A0
:102B5000420708D5CA0706D0256804222A62E26F18
:102B600042F00202E26702070ED503F0200201F0F4
:102B700080552A4352EAC17206D0256808222A628B
:102B8000E26F42F00802E267E26F002A3AD0800664
:102B900008D503F0200001F08051084302D0204600
:102BA00001F0F4FBE06F000703D420688068400662
:102BB0002AD5204601F0DCFB2068816849061ED535
:102BC000816821F040018160606FC0B12D490165CD
:102BD000606FFDF75FFF002814D0606F016DBDE8E6
:102BE00070400847850615D503F0200501F0805692
:102BF00035430FD02046BDE8704001F0C7BB2046EA
:102C0000FFF77BFF70BD05E02046FFF776FF002051
:102C1000E067F7E7C6024FF020050CD54E020AD553
:102C2000E803106284F8795084F87A502046BDE8B1
:102C30007040FFF761BF06060AD503F0800601F475
:102C400000010E4304D02046BDE8704001F02EBEC6
:102C500041060BD5590609D51168204621F04001DF
:102C6000116084F8795000F005F9CBE70002C9D56E
:102C70005800C7D5106820F080401060C2E70000FF
:102C8000010000105D43000810B5040003D094F863
:102C9000790010B107E0012010BD002084F8780011
:102CA000204600F027F8242084F879002068016885
:102CB00021F001010160204601F0A4FB0128EBD0C6
:102CC000606B10B1204601F0B7FA2068416821F42A
:102CD000904141602068816821F02A01816020686C
:102CE000016841F0010101602046BDE8104001F09B
:102CF00007BB000010B5006886B01B49884230D180
:102D00001A48016841F001010160006800F001000B
:102D1000059016481030016841F01001016000680C
:102D20000121134C00F0100005904FF4007000904A
:102D30000220CDE901010390072069460490204656
:102D4000FDF7FAFE4FF48061204600916946FDF7D9
:102D5000F3FE2520FEF779F8032225201146FEF721
:102D600081F806B010BD000000100140E044025898
:102D70000000025890F87A30202B4CD1B9B1B2B192
:102D800090F87830012B46D0012380F878304166E6
:102D9000A0F86820A0F86A20FF228168B1F5805F62
:102DA00007D07F2351B1B1F1805F0CD010E001203A
:102DB0007047016921B940F2FF1107E0016909BBC1
:102DC000A0F86C2004E00169E1B13F21A0F86C108B
:102DD0000021C167222280F87A2080F878100168EB
:102DE0008A6842F001028A6001680A6892000CD584
:102DF0000A6842F480720A600068816841F080517C
:102E0000816006E0A0F86C30E2E7086840F490705A
:102E100008600020704702207047000030B500684D
:102E2000114988420CD1114A5088010408D4114636
:102E30004FF000034404097806D50A2901D05380D5
:102E400030BD40F400400DE00D2909D0084DC0F31D
:102E50000D04401C80B2C72829555080EFD830BDE2
:102E600040F48040508030BD001001401400002428
:102E7000500000247047FEE7144870B586B0016822
:102E800041F004010160016801F00401059101684D
:102E900041F010010160006800260325694600F03A
:102EA0001000059008200124CDE900060848CDE96E
:102EB0000245FDF741FE20206946CDE900060548A0
:102EC000CDE90245FDF738FE06B070BDE04402587A
:102ED00000100258000802582DE9F0411C4C012551
:102EE0001C4E01281C4F12D0207848B108213046D2
:102EF000FDF716FF68B120213846FDF711FF40B1FC
:102F000008213046FDF70CFF012817D01DE0257081
:102F1000ECE70A2001F074FD002020700821304603
:102F2000FDF7FEFE28B120213846FDF7F9FE18B165
:102F30000BE00120BDE8F0810220FBE720213846AC
:102F4000FDF7EEFE012800D125700020F2E7000019
:102F50002400002400100258000802582DE9F04116
:102F60000D4F00240646214620467B883A8800F013
:102F7000E1F93D88002178884543084600F0C6F90C
:102F800000F0C0FA03E0304600F066FA641CAC4280
:102F9000F9D3BDE8F08100006C1200242DE9F04166
:102FA0001E490027F0222C242A252B264FF4A0733B
:102FB00038B1012817D002284FF0010C1BD003288C
:102FC00022D08F710A804B800C8100244D818E812C
:102FD0004B880A880021084600F0ACF92046BDE87D
:102FE000F04100F081B98F710B804A800C8101247F
:102FF0004D818E81ECE781F806C00A804B800C8100
:1030000002244D818E81E3E781F806C00B804A805F
:103010000C8103244D818E81DAE700006C120024BC
:103020002DE9F0410B4C16460F460546608900F02D
:103030004DFA284600F010FAA08900F047FA384609
:1030400000F00AFA208900F041FA3046BDE8F0416C
:1030500000F002BA6C1200242DE9F0415C1A151A36
:10306000641C069F6D1CA3B2AAB200F063F90B4E5C
:10307000308900F02BFA654300F044FA002403E0A5
:10308000384600F0E9F9641CAC42F9D97388002194
:1030900032880846BDE8F04100F04CB96C120024BB
:1030A0001A4810B586B0016841F00201016000685D
:1030B0006946174C00F00200059041F203000090B1
:1030C000012001900290032003902046FDF734FD7B
:1030D000012220461146FDF72CFE01222046022146
:1030E000FDF727FE012220461103FDF722FE00F026
:1030F0007BFEA00400F0B6FE00F00CF80122204692
:103100001146FDF716FE06B010BD0000E04402585F
:103110000004025870B50A4D4FF480440022214645
:103120002846FDF706FE322001F06AFC0122214606
:103130002846FDF7FEFDBDE870401E2001F060BC92
:103140000004025810B5FFF7ABFF00F07BF9322006
:1031500001F056FC362000F0B9F9002000F09AF991
:103160003A2000F0B3F9052000F094F9B22000F005
:10317000ADF90C2000F08EF90C2000F08BF9002046
:1031800000F088F9332000F085F9332000F082F94F
:10319000B72000F09BF9352000F07CF9BB2000F04F
:1031A00095F9192000F076F9C02000F08FF92C2055
:1031B00000F070F9C22000F089F9012000F06AF9EE
:1031C000C32000F083F9122000F064F9C42000F05D
:1031D0007DF9202000F05EF9C62000F077F90F207D
:1031E00000F058F9D02000F071F9A42000F052F955
:1031F000A12000F04FF9E02000F068F9D02000F0A5
:1032000049F9042000F046F90D2000F043F911209F
:1032100000F040F9132000F03DF92B2000F03AF9BE
:103220003F2000F037F9542000F034F94C2000F032
:1032300031F9182000F02EF90D2000F02BF90B20A9
:1032400000F028F91F2000F025F9232000F022F9D2
:10325000E12000F03BF9D02000F01CF9042000F040
:1032600019F90C2000F016F9112000F013F91320C1
:1032700000F010F92C2000F00DF93F2000F00AF9C1
:10328000442000F007F9512000F004F92F2000F04D
:1032900001F91F2000F0FEF81F2000F0FBF82020AD
:1032A00000F0F8F8232000F0F5F8212000F00EF9E6
:1032B000112000F00BF9782001F0A2FB292000F08A
:1032C00005F9C82001F09CFB0020FFF767FE0122F2
:1032D00004481146FDF72DFDBDE810404FF6FF7084
:1032E000FFF73CBE00040258002158B1012804D069
:1032F000022804D0032805D103E0602102E0C021A8
:1033000000E0A021362000F003B9000070B5084CA1
:103310000D460646608900F0D9F8304600F09CF86A
:10332000A08900F0D3F82846BDE8704000F094B8BA
:103330006C1200242DE9F04104460E4F10448846DB
:10334000401E86B2C818401E85B2788900F0BEF8CB
:10335000204600F081F8304600F07EF8B88900F091
:10336000B5F8404600F078F82846BDE8F04100F096
:1033700073B800006C1200242DE9F84F1F460C466C
:1033800082468B46580700D00120790800EBD70011
:10339000203A10FB01F0002602F0FF09C0B20090B5
:1033A00040E00C2F0FD0102F11D0182F3DD1204905
:1033B00009EBC90001EB80004FF00008855D28068D
:1033C00009D50A9A0BE01B4909EB4900F2E71A49B3
:1033D00001EB0910F0E70B9828B9184842882146FC
:1033E0005046FFF71DFE6806641C050E1448A4B283
:1033F0004088A04219D9A4EB0B00B84209D10AF1C8
:1034000001005C461FFA80FA0D48018851450CD92D
:1034100006E008F1010000F0FF08B8F1080FCED374
:10342000761CF6B200988642BBD3BDE8F88F000048
:103430009A570008364D0008AA5100082A000024B7
:103440006C120024012010B500F040F8BDE81040D7
:10345000322001F0D5BA000070B50D4E4FF4805502
:103460000022044629463046FDF763FC012230461F
:103470000221FDF75EFC200A00F0E4FCE0B200F05F
:10348000E1FC29463046BDE870400122FDF751BC01
:103490000004025870B50C4D4FF4805400220646CB
:1034A00021462846FDF745FC012228460221FDF76A
:1034B00040FC304600F0C6FC21462846BDE870407E
:1034C0000122FDF736BC00000004025870B50C4E16
:1034D0004FF480550022044629463046FDF729FC6A
:1034E000002230460221FDF724FCE0B200F0AAFCE5
:1034F00029463046BDE870400122FDF71ABC0000A5
:103500000004025801480089FFF7E0BF6C12002454
:1035100010B50C46FFF7DAFFE0B2BDE81040FFF748
:10352000B9BF00000E4810B586B0016841F0010136
:103530000160006869460B4C00F001000590022014
:103540000090012001900290032003902046FDF797
:10355000F3FA012220460221FDF7EBFB06B010BD75
:10356000E0440258000002580EB5002101200090EE
:103570000323CDE9010112210246480600F001F8BB
:103580000EBD2DE9FF4707461E460CA814460D4602
:1035900090E80007FDF738FC01208DF800000020BE
:1035A0008DF808508DF80C008DF809008DF80D800D
:1035B0008DF80A0068468DF80E908DF8014001974D
:1035C0008DF80B608DF80FA0FDF7F4FB0420FDF7DC
:1035D00029FC04B00020BDE8F087704710B5040353
:1035E00000F0E6F800F08EF8002321462F2220207C
:1035F00000F05EFABDE8104000F084B808B500F0B5
:1036000023FA00F01BF800F041F80B494880A0F5C0
:103610006F4116390ED100F0CBF80023C3221946B2
:10362000C02000F045FA30208DF8000001216846E6
:1036300000F0B4FA08BD000026000024022010B5F6
:1036400000F03CF80446800706D400F0B1F80220F0
:1036500044F0020100F0EEF8002301221946382060
:1036600000F026FA01490120087010BD2600002450
:1036700070B508231546EF2204460B2000F018FA17
:1036800029462046BDE8704000F000BA0A4808B557
:103690004FF00003007808B1EF2200E0652200211E
:1036A000902000F005FA0221684600F0EFF9BDF81D
:1036B000000040BA08BD00002600002408B5002123
:1036C00001288DF8001003D0022803D0032803D06E
:1036D000052002E0352000E0152009494FF00003E5
:1036E000097809B1C32200E04122002100F0E0F98D
:1036F0000121684600F0CAF99DF8000008BD0000ED
:103700002600002410B50120FFF7D8FFC007FAD12A
:1037100010BD00002DE9F05FC1F30B06DFF88C80CF
:103720000F0B8A46C6F580548146A242154600D842
:103730001446404639034FF480528B46FFF798FFFA
:10374000002006E0321818F80210FF2903D1401CAF
:1037500080B2A042F6D3A04221D23846FFF73EFF06
:10376000002006E0831919F80020401C80B208F8F8
:103770000320A042F6D34FF480525946404600F051
:1037800025F8A5420FD0281BA144A24485B20026EB
:103790007F1C4FF48054A542CBD82C46C9E7224663
:1037A00051464846EBE7BDE8F09F0000E4010024E5
:1037B00005484FF00003007808B1032200E0012221
:1037C0000021062000F074B9260000242DE9F04104
:1037D00007460E46C8B21546C0F58074A24200D80E
:1037E00014464FF4807822463146384600F00DF8F2
:1037F000A54208D0281B27442644444685B2A5424A
:10380000F1D82C46EFE7BDE8F08170B516460C46BE
:103810000546FFF7CDFF00232146EF22022000F0EE
:1038200047F93146284600F0B9F9BDE87040FFF786
:1038300069BF000013B5012804D0022809D003286D
:1038400009D0012009494FF00003097829B1C322AA
:1038500004E03120F6E71120F4E74122002100F0D6
:1038600027F9012101A800F099F91CBD26000024C8
:103870007047F0B54B6A4FF040652BB1AA4203D0B8
:1038800004688B6A5B1E23614FF4F8038C69002C7B
:1038900072D00E6ACEB306688C68F461CC69F4B15C
:1038A000D1E90B67D1F824C093FAA3F33E434F6BE1
:1038B000B3FA83F347EA0C073E434F699F400B6915
:1038C0003E431E430B6A1E43CB681E438B6926434F
:1038D0001E430B686FE0006849688161F0BDD1E963
:1038E0000B454E6A93FAA3F32C434D6BB3FA83F363
:1038F00035432C434D699D400B692C431C430B6A97
:103900001C438B6909681C436AE0FFE7CE690EB36C
:10391000D1E90B7CD1F824E093FAA3F347EA0C0732
:10392000D1F834C0B3FA83F34CEA0E0C47EA0C0723
:10393000D1F814C00CFA03FCCB6847EA0C071F430C
:103940000B68374327431F43036817435F61AA424D
:10395000C1D1F0BDD1E90B564F6A93FAA3F33543B9
:103960004E6BB3FA83F33E4335434E6909689E407C
:103970003543254362E0FFE70C6AB4B306688C6800
:10398000F461CC69CCB1D1E90B67D1F824C093FACA
:10399000A3F33E434F6BB3FA83F347EA0C073E436E
:1039A0004F699F400B693E431E430B6A1E43CB6821
:1039B0001E438B6926431E432DE0D1E90B454E6A19
:1039C00093FAA3F32C434D6BB3FA83F335432C43A3
:1039D0004D699D400B692C431C430B6A89691C434C
:1039E00000680C4314434461F0BDFFE7CC69B4B1F7
:1039F000D1E90B67D1F824C093FAA3F33E434F6B90
:103A0000B3FA83F347EA0C073E434F699F40CB6804
:103A10003E431E432643036816435E6197E74C6AA4
:103A2000002CE1D0D1E90B5693FAA3F335434E6B4A
:103A30004969B3FA83F326433543994000680D433F
:103A400015434561D0E700000F480E4910B50160ED
:103A500001214160042181601021C160C90491FAF3
:103A6000A1F1B1FA81F1491E01614FF48061416118
:103A700000218161C1610162FDF76AFA002800D06E
:103A8000012010BD0050005298010024074A491E31
:103A900010B51268116141F2883201460348FDF702
:103AA00027FB002800D0012010BD00009801002451
:103AB00000B58FB00593CDE9000191074FF00000EC
:103AC00009D002F00301012907D0022908D0D1430F
:103AD000890708D00AE0069008E04FF4807104E0FE
:103AE0004FF4007101E04FF440710691910889078D
:103AF0000AD0C2F38101012908D0022909D06FEA56
:103B00009201890708D00AE0079008E04FF480612D
:103B100004E04FF4006101E04FF4406107911109A6
:103B200089070AD0C2F30111012908D0022909D05E
:103B30006FEA1211890708D00AE0039008E04FF4F9
:103B4000805104E04FF4005101E04FF440510391E3
:103B5000910905D00121B1EB921F03D109060DE0B7
:103B600009900CE00221B1EB921F01D1090605E09A
:103B70006FEA9211890702D14FF0407109910D90BF
:103B800041F28832089069460B900C900248FDF78C
:103B90009BF90FB000BD000098010024074A491EA0
:103BA00010B51268116141F2883201460348FDF7F1
:103BB000FDFA002800D0012010BD0000980100246B
:103BC0002DE9F0411E46174688460546069C11E041
:103BD000601C0FD024B1FDF7B1F8801BA04209D9B9
:103BE000042085F84100686C40F001006864012001
:103BF000BDE8F0812868806810EA080000D0012044
:103C0000B842E5D10020F3E72DE9F047DFF8E48082
:103C100004460F464FF00009D8F80000C043800763
:103C200009D0344D283D286820F080602860FDF7D9
:103C300085F8064607E00120BDE8F087FDF77EF82D
:103C4000801B02284ED828680001F7D4D8F800104D
:103C5000226821F47C3141EA0231C8F80010207A50
:103C60004FF4FE02A1884002491EA0F5007080B208
:103C7000C1F308010843A189491E02EA0141084332
:103C8000217C1202491E02EA0161084319491031E0
:103C900008601848001D0168626921F0C0011143E5
:103CA00001600168A26921F02001114301606FB138
:103CB0000168012F0ED041F400110160286840F026
:103CC00080602860FDF73AF804460DE0016841F491
:103CD0000021F2E741F48011EFE7FDF72FF8001B18
:103CE000022801D90320A7E728680001F5D5484636
:103CF000A2E70000284402582DE9F047DFF8E480ED
:103D000004460F464FF00009D8F80000C043800772
:103D100009D0344D283D286820F080502860FDF7F8
:103D20000DF8064607E00120BDE8F087FDF706F82C
:103D3000801B02284ED828688000F7D4D8F80010DD
:103D4000228821F07C7141EA0251C8F80010207AE3
:103D50004FF4FE02A1884002491EA0F5007080B217
:103D6000C1F308010843A189491E02EA0141084341
:103D7000217C1202491E02EA0161084319491831E7
:103D800008601848001D0168626921F44061114310
:103D900001600168A26921F40071114301606FB1F3
:103DA0000168012F0ED041F080710160286840F059
:103DB00080502860FCF7C2FF04460DE0016841F422
:103DC0008001F2E741F40001EFE7FCF7B7FF001BC9
:103DD000022801D90320A7E728688000F5D54846C6
:103DE000A2E700002844025810B5154C07211348DB
:103DF0004FF0007204F1080320604FF4800060600F
:103E0000002083E80700521062619200A261CA0795
:103E1000606362650A07C4E907206062C4E90A01B9
:103E20002046FEF79BFB2068016841F0010101601C
:103E3000BDE81040FF2000F005B800000038004049
:103E4000E411002401B582B04FF47A700123009090
:103E500001AA034802A9FEF7A3FC9DF804000EBDC9
:103E6000E41100240A4A11680B6823F001030B6077
:103E700011688B6823F0E0438B6011688B68034303
:103E80008B601068016841F001010160704700001B
:103E9000E411002410B502685169936943F00803E6
:103EA00093610268936943F0100393610268136899
:103EB00023F0010313600268136940F26B34A343DB
:103EC00013610268936823F44043936090F8812063
:103ED000042A0CD08A060AD5D0F8842042F0800249
:103EE000C0F884200268936943F02003936190F83E
:103EF0008120032A1DD04A060AD5D0F8842042F03A
:103F00000402C0F884200268936943F0400393617F
:103F1000826AB2F5800F0CD10A060AD5D0F8842047
:103F200042F00202C0F884200268936943F08003E3
:103F300093618A050AD5D0F8842042F00102C0F8C6
:103F400084200268936943F400739361C9050AD51C
:103F5000D0F8841041F00801C0F8841001688A6923
:103F600042F480728A610021A0F86210A0F86A1001
:103F700010BD2DE9F0411E4617460D468046069CB1
:103F80000AE0601C08D024B1FCF7D8FE801BA042D8
:103F900002D90320BDE8F081D8F80000406935EA75
:103FA000000004D00020B842EBD00020F2E701204E
:103FB000F9E770472DE9F04F93B01F4615468A4642
:103FC00004468146580700D0012000EBD7000C2F93
:103FD00010FB07F0C0B2129003D0102F01D0182FA1
:103FE0002FD1024669462846FCF72AFD002024E02E
:103FF0001DF808600025DFF850B0300601D51C9A86
:1040000003E01D9828B9BBF8002051462046FFF771
:1040100007F87006641CA4B2060EA4EB0900B842AF
:1040200004D10AF101004C461FFA80FA6D1CEDB272
:10403000082DE2D308F10100C0B2129980468842EF
:10404000D6D313B0BDE8F08F2C0000242DE9FF4F2C
:1040500083B09B460E46044680468A46DDE91075CD
:10406000002081461FE0B9F1000F22D005994FF0E2
:10407000000908EB0100401BA04202DA7019444617
:1040800086B20AEB0B00401BB0420FDBDDE91201E8
:104090002B463A46CDE9000131462046FFF78AFF1C
:1040A000601984B2BF1C3A78002ADCD107B0BDE8A1
:1040B000F08F802A01D90120D3E7059908EB010090
:1040C000A0EB5500A04202DA7019444686B20AEB12
:1040D0000B00401BB042E9DB0D2A0DD0DDE91201D7
:1040E0002B46CDE9000131462046FFF745F904EBA8
:1040F000550084B27F1CD6E77019444686B27F1CF7
:10410000F5E7000070B5284C9CB0256825F0040543
:104110002560254C00260C34256845F44045256073
:10412000256805F440451B952568AD04FCD50124A0
:1041300000940CAD03962404019402240994CDE963
:104140000A410796082485E80D00CDE91046684627
:10415000FDF7B6FF88B93F2013900320CDE9140680
:1041600040200101CDE91640CDE9180150201A90F8
:10417000022113A8FDF7F6FD10B101201CB070BD9F
:104180000A48016841F0800101600848F430016884
:1041900041F002010160006800F002001B90FCF792
:1041A000C3FC0020EAE700000C4802580044025813
:1041B000FCF7CABD1C48016841F4700101601B494D
:1041C000086840F001000860184A002010321060B2
:1041D0000A68174B1A400A60144A18321060121D00
:1041E0001060121D1060114A28321060121D1060FC
:1041F000121D1060121D1060121D1060121D106043
:10420000121D1060121D10600A6822F480220A60DC
:1042100006496031086001200649C1F80801C0065E
:10422000014980390860704788ED00E00044025879
:104230007FEDF6EA0080005190F83410C90706D0EF
:1042400001684A68836B22F400321A434A6090F88E
:104250003410890706D501684A68C36B22F480329E
:104260001A434A6090F83410490706D501684A6835
:10427000036C22F480221A434A6090F83410090734
:1042800006D501684A68436C22F400421A434A602A
:1042900090F83410C90606D501688A68836C22F448
:1042A00080521A438A6090F83410890606D5016856
:1042B0008A68C36C22F400521A438A6090F8341062
:1042C000490611D501684A68036D22F480121A4329
:1042D0004A60016DB1F5801F06D101684A68436DDF
:1042E00022F4C0021A434A6090F83410090606D539
:1042F00001684A68806D22F4002202434A607047D8
:10430000F8B500250446C567FCF718FD0746206888
:1043100000686FF07E46000708D500223B464FF448
:1043200000112046009600F0FBFA60B92068006892
:1043300040070AD500223B464FF4800120460096F4
:1043400000F0EEFA08B10320F8BD202084F87900CF
:1043500084F87A00002084F87850F8BD10B5806B9E
:104360000021A0F86A10A0F86210FEF7C6FB10BD8D
:1043700001680A6822F490720A6001688A6822F073
:1043800001028A60202180F87A10704710B5B0F8D9
:104390006C2090F87A300168222B05D0088B40F011
:1043A00008000883022010BD898C8368B3F5805F04
:1043B00001D103696BB11140426E531C4366117009
:1043C000B0F86A10491E0904090CA0F86A1007D059
:1043D00015E0436E11401980416E891C4166EFE77C
:1043E00001680A6822F490720A6001688A6822F003
:1043F00001028A60202180F87A10FEF70FFD00206C
:1044000010BD00002DE9F04F044600688025FD4BEB
:104410000021D4F810C087B0A6680F46D4F81C80DD
:1044200046EA0C06D4F814C0A26A4CEA080C46EA24
:104430000C0632430668DFF8D0C306EA0C061643C2
:10444000066020684268E66822F4405232434260C7
:104450002268A0699A4201D0266A3043A66AB6F162
:10446000005F04D1D4E90B6C46EA0C063043966831
:10447000DFF898C306EA0C06064396602068C26A15
:10448000666A22F00F023243C262E14E2068E14ABE
:10449000B04210D1126802F03802182A74D005DC3C
:1044A000CAB3082A7AD0102A47D179E0202A7BD0D3
:1044B000282A7CD17AE0D84EB04209D1126802F0A5
:1044C0000702062A73D2DFE802F053696B6D6F7141
:1044D000D24EB04209D1126802F00702062A66D213
:1044E000DFE802F0465C5E606264CD4EB04209D106
:1044F000126802F00702062A59D2DFE802F0394FAB
:1045000051535557C74EB0420BD1126802F0070203
:10451000062A4CD200E00EE0DFE802F02A404244D6
:104520004648C14EB04209D1126802F03802182A3A
:1045300038D0BBDCB4E74FF0010538E0BB4EB042E9
:1045400009D1126802F00702062A30D2DFE802F031
:104550001026282A2C2EB64EB0420BD1126802F03B
:104560000702062A23D2DFE802F003191B1D1F21D0
:1045700000251CE098421AD1A64A121D126802F0CA
:104580000702062A13D202E00CE007E00CE0DFE8A5
:1045900002F0030507090B0D022508E0042506E0DB
:1045A000402504E0082502E0102500E02025DFF882
:1045B00064B2A04E9842DFF880A2ABF1540B73D1E5
:1045C000102D31D006DC022D09D0042D0AD0082D83
:1045D0002FD111E0202D29D0402D2AD107E0FCF762
:1045E00057FE13E06846FCF769FE01980EE003A849
:1045F000FCF7E2FE049809E0DBF800105846890653
:1046000010D50068C0F3C1012AFA01F0002811D0CA
:104610006168894601EB410181420AD8B0EB093F4C
:1046200007D808E05046F3E78448F1E74FF400402C
:10463000EEE7012733E1102D4FF000084ED006DCE5
:10464000022D0FD0042D15D0082D04D12DE0202DE2
:104650004AD0402D13D00127794AA0F540719142EC
:1046600070D9E6E7FCF714FE626A0023414636F88B
:1046700012200DE06846FCF721FE019803E003A834
:10468000FCF79AFE04980023616A36F81120194657
:10469000FBF773FE62680902030241EA10615008E9
:1046A000181841EB080115E032E0DBF8001058461D
:1046B000890609D500680023C0F3C1012AFA01F078
:1046C000616A36F8112015E0606A002336F8102080
:1046D00050460FE00023FBF750FEBDE7606A002361
:1046E00036F81020554805E0606A002336F810209F
:1046F0004FF400400021FBF740FE0902020241EAAC
:1047000010614FEA590010184A4641EB0801E1E7F1
:10471000E3694FF4004293424DD1082D23D005DCCC
:104720008DB1012D12D0042D06D112E0102D35D0FF
:10473000202D3AD0402D11D0012721F00F00C1F3D8
:10474000420108435AE0FDF713FC16E0FDF726FC92
:1047500013E06846FCF7B2FD01980EE003A8FCF7F1
:104760002BFE049809E0DBF800105846890608D5AE
:104770000068C0F3C1012AFA01F0616A36F811102D
:1047800010E0606A36F81010BAFBF1F04100606882
:1047900001EB5001B1FBF0F081B2CEE7606A36F870
:1047A00010102648B0FBF1F0F0E7606A36F8100010
:1047B000B2FBF0F0EAE7082D4AD00ADC0DB3012D78
:1047C00043D0042D7FF44DAF6846FCF777FD019888
:1047D00009E0102D52D0202D55D0402DF2D103A844
:1047E000FCF7EAFD0498616A36F81110B0FBF1F1AC
:1047F000606801EB5001B1FBF0F080B22168C86045
:104800004DE01FE0000C0058F369FFCFFFF4FF11EB
:104810000010014054440258004400400048004049
:10482000004C00400050004000140140007800405F
:10483000007C00401E4D00080090D00300093D00A0
:10484000FFFC0F00FDF794FBCDE7FDF7A7FBCAE7E0
:10485000DBF80020594692060AD50968C1F3C10267
:104860002AFA02F1626A36F81220B1FBF2F20FE086
:10487000616A36F81120BAFBF2F209E0616A36F893
:1048800011200949F1E7616A36F81110B2FBF1F223
:10489000616802EB5102B2FBF1F189B2C16007B06D
:1048A0003846BDE8F08F000000093D0090F879100F
:1048B000212901D002207047B0F8621021B181682F
:1048C000B1F5805F13D014E001680A68920004D546
:1048D0008A6822F400028A6003E00A6822F08002FB
:1048E0000A600068016841F0400101600CE0016964
:1048F00061B1C16D4A1CC265026809781185B0F8C2
:104900006210491EA0F8621000207047C16D026855
:104910000988C1F308011185C16D891CC165EEE7E5
:104920002DE9F0411E46174688460446069D1CE0C8
:10493000681C1AD025B1FCF701FA801BA84214D9D3
:104940002068016821F4D07101602068816821F03D
:1049500001018160202084F8790084F87A00002029
:1049600084F878000320BDE8F0812068C16938EA46
:10497000010004D00020B842DAD00020F3E7012083
:10498000F9E7000070B50D4D00240D48FEF7BCF8A6
:1049900002E0641CAC4204D80948FEF7AFF82028B6
:1049A000F7D1002402E0641CAC4206D8054901227C
:1049B0000348FEF7DFF90028F5D170BDFFFF0100C5
:1049C0001801002414000024FEE70907090E00283E
:1049D00004DB00F1E02080F80014704700F00F00C5
:1049E00000F1E02080F8141D7047704710B50446B0
:1049F0000420FEF761F80148046010BD1000002497
:104A000070B5002405464FF47A7603E0304600F096
:104A100005F8641CAC42F9D370BD000070B54FF0CE
:104A2000E02500216C69094AAB6912685043AA6904
:104A30009A42FCD002D2A3EB020302E0A4EB0206EE
:104A40003344194413468142F1D370BD1000002451
:104A500008B5FBF741FDFCF77FF90423022205218D
:104A6000A020FFF74FFB4FF4C870FFF7BFFF4FF4D4
:104A7000E13000F01FF9FEF755FDFEF7FDF9FEF7F6
:104A800073FDFEF75FFBFBF791FE4FF6FF752846BF
:104A9000FEF764FA10214FF47846084644A33246E4
:104AA000FBF7C6FD1F222021102047A3FBF7C0FD06
:104AB0001F223021102049A3FBF7BAFD40213246C6
:104AC00010204BA3FBF7B4FDFEF798FDDFF834810F
:104AD0004FF4FA744EF6167715E01F22602110206D
:104AE00049A3FBF7A5FD2046FFF78AFF1F2260219F
:104AF00010204BA3FBF79CFD2046FFF781FF02210E
:104B00004046FCF712F9FEF7C1FDB842E5D11F227D
:104B10006021102048A3FBF78BFD4B4C0020FEF7D3
:104B2000DBF90128607018D1EF2240F23F137021A9
:104B300000950020FEF790FA1F227021102043A359
:104B4000FBF776FD227847486168FEF7E3FD1F22F8
:104B50007021102044A3FBF76BFD6078022816D16A
:104B60001F227021102046A3FBF762FD22784A48DD
:104B70006168FEF77DFD1F227021102047A3FBF71F
:104B800057FD454B802110203246FBF751FD6088D0
:104B9000401C60800A20FFF733FF60881428BDD1D5
:104BA00002214046FCF7C1F800206080B6E7000013
:104BB0002053544D3332483720573235513634283C
:104BC00051535049292020002020C7B6C8EBCABD48
:104BD000BFAAB7A2CDF8202020000000206D637589
:104BE0006465762E74616F62616F2E636F6D000075
:104BF000204B313A577269746520204B323A526526
:104C000061640000000002585732355136342043A9
:104C10006865636B204661696C6564210000000073
:104C2000506C6561736520436865636B21202020AB
:104C300020202020200000005732355136342052E9
:104C400065616479210000000000002453746172E2
:104C500074205772697465205732355136342E2EC0
:104C60002E2E0000F64C00085732355136342057AE
:104C7000726974652046696E697368656421000015
:104C80005374617274205265616420573235513615
:104C9000342E2E2E2E200000300000245468652073
:104CA00044617461205265616465642049733A20EF
:104CB000202000000B490A4A10B5C1E9002000205D
:104CC0008860C860086188610C2048610846FDF76B
:104CD000DBFFBDE81040044901220248FEF74AB854
:104CE0000010014018010024140000244FF040700F
:104CF000E1EE100A7047573235513634204368656B
:104D0000636B3A204F4B204F4B204F4B000000006D
:104D10000000010203040102030406070809010060
:104D200002000400060008000A000C001000200029
:104D300040008000000100000000000000000000B2
:104D40000000000000003F400000000000000000E4
:104D50003000400030004000000009000BC03D0062
:104D60000BC03D00090018C024407FE02240318084
:104D70000000180024C01B000D8032400180038019
:104D80001C4027401C8007400040100060000000CD
:104D90000000000000000000000000001F80204014
:104DA00040200000402020401F800000000009003B
:104DB00006001F80060009000000040004003F8078
:104DC000040004000000001000600000000000006B
:104DD00000000400040004000400040000000000BF
:104DE00000400000000000000000002001C006009C
:104DF0003800400000001F802040204020401F80DD
:104E00000000000010403FC000400000000018C03B
:104E100021402240244018400000108020402440BF
:104E200024401B80000002000D0011003FC0014023
:104E300000003C80244024402440238000001F8048
:104E4000244024403440038000003000200027C06C
:104E50003800200000001B802440244024401B8098
:104E600000001C0022C0224022401F8000000000E1
:104E70000000084000000000000000000000046086
:104E8000000000000000000004000A001100208063
:104E90004040090009000900090009000000000065
:104EA0004040208011000A00040018002000234028
:104EB0002400180000001F802040274029401F4088
:104EC0000000004007C039000F0001C00040204032
:104ED0003FC0244024401B8000001F802040204011
:104EE00020403080000020403FC0204020401F80F4
:104EF000000020403FC024402E4030C00000204031
:104F00003FC024402E00300000000F0010802040E1
:104F100022403380020020403FC0040004003FC014
:104F20002040204020403FC0204020400000006042
:104F3000202020203FC02000200020403FC02440EF
:104F40000B0030C0204020403FC0204000400040C7
:104F500000C03FC03C0003C03C003FC000002040F8
:104F60003FC00C4023003FC020001F802040204055
:104F700020401F80000020403FC024402400180033
:104F800000001F802140214020E01FA000002040A1
:104F90003FC02440260019C0004018C024402440CF
:104FA000224031800000300020403FC020403000CF
:104FB000000020003F80004000403F802000200093
:104FC0003E0001C0070038002000380007C03C0048
:104FD00007C038000000204039C0060039C020401A
:104FE00000002000384007C038402000000030405A
:104FF00021C02640384020C00000000000007FE0B3
:10500000402040200000000070000C0003800040A1
:1050100000000000402040207FE000000000000071
:1050200020004000200000000000001000100010D0
:105030000010001000100000000040000000000000
:105040000000000002800540054003C00040200031
:105050003FC004400440038000000000038004407F
:1050600004400640000000000380044024403FC08C
:1050700000400000038005400540034000000000A0
:1050800004401FC0244024402000000002E00550DE
:1050900005500650042020403FC00440040003C0D7
:1050A00000400000044027C0004000000000001045
:1050B0000010041027E00000000020403FC0014025
:1050C000070004C00440204020403FC00040004092
:1050D000000007C0040007C0040003C00000044033
:1050E00007C00440040003C00040000003800440E7
:1050F000044003800000041007F0045004400380C3
:105100000000000003800440045007F00010044039
:1051100007C00240040004000000000006400540F3
:10512000054004C00000000004001F80044000404F
:105130000000040007800040044007C00040040055
:10514000070004C0018006000400060001C007003B
:1051500001C006000000044006C0010006C0044073
:1051600000000410071004E00180060004000000A5
:10517000044005C006400440000000000000040098
:105180007BE040200000000000000000FFF0000075
:105190000000000040207BE0040000000000400010
:1051A00080004000200020004000000000000000BF
:1051B00000000000000000000000000000000000EF
:1051C0001FCC000C000000000000000008003000B0
:1051D00060000800300060000000022003FC1E2078
:1051E000022003FC1E200220000000000E18110403
:1051F0003FFF10840C78000000000F0010840F386F
:1052000000C0077818840078000000780F8410C46C
:1052100011240E9800E40084000808006800700063
:10522000000000000000000000000000000000007E
:1052300007E018182004400200000000400220048B
:10524000181807E000000000000002400240018042
:105250000FF00180024002400000008000800080CA
:105260000FF800800080008000000001000D000E9B
:10527000000000000000000000000000008000802E
:10528000008000800080008000800000000C000C86
:1052900000000000000000000000000000060018F0
:1052A00000600180060018002000000007F00808D8
:1052B00010041004080807F00000000008040804A7
:1052C0001FFC000400040000000000000E0C10147D
:1052D0001024104411840E0C000000000C1810045F
:1052E0001104110412880C700000000000E003207B
:1052F000042408241FFC0024000000001F981084D0
:1053000011041104108810700000000007F00888D4
:105310001104110418880070000000001C00100027
:1053200010FC13001C001000000000000E38114497
:105330001084108411440E38000000000700088C0F
:1053400010441044088807F000000000000000002E
:10535000030C030C0000000000000000000000012E
:105360000106000000000000000000000080014075
:10537000022004100808100400000220022002206D
:105380000220022002200220000000001004080871
:105390000410022001400080000000000E001200F6
:1053A000100C106C10800F00000003E00C1813E4C8
:1053B000142417C4082807D000000004003C03C4CC
:1053C0001C40074000E4001C000410041FFC1104F2
:1053D000110411040E880070000003E00C18100482
:1053E0001004100410081C10000010041FFC10040E
:1053F00010041004080807F0000010041FFC11043A
:10540000110417C410040818000010041FFC110434
:10541000110017C010000800000003E00C18100471
:10542000100410441C780040000010041FFC10847D
:105430000080008010841FFC100400001004100481
:105440001FFC100410040000000000030001100104
:1054500010011FFE10001000000010041FFC1104BA
:1054600003801464181C1004000010041FFC1004B6
:10547000000400040004000C000010041FFC1F00C6
:1054800000FC1F001FFC1004000010041FFC0C0493
:10549000030000E010181FFC100007F008081004BB
:1054A00010041004080807F0000010041FFC10840A
:1054B0001080108010800F00000007F008181024E2
:1054C0001024101C080A07F2000010041FFC11042D
:1054D000110011C011300E0C000400000E1C11044C
:1054E0001084108410441C380000180010001004B0
:1054F0001FFC100410001800000010001FF810041A
:105500000004000410041FF8100010001E0011E039
:10551000001C007013801C0010001FC0103C00E035
:105520001F0000E0103C1FC000001004180C1634CF
:1055300001C001C01634180C100410001C00130424
:1055400000FC13041C00100000000804101C106470
:10555000108413041C041018000000000000000058
:105560007FFE4002400240020000000030000C00BC
:1055700003800060001C00030000000040024002A5
:1055800040027FFE0000000000000000000020003C
:105590004000400040002000000000010001000128
:1055A0000001000100010001000100004000400076
:1055B000200000000000000000000000009801240E
:1055C00001440144014400FC000410001FFC008859
:1055D00001040104008800700000000000700088D1
:1055E000010401040104008800000000007000882C
:1055F0000104010411081FFC0004000000F801442C
:1056000001440144014400C80000000001040104F9
:105610000FFC1104110411001800000000D601292C
:105620000129012901C90106000010041FFC0084A2
:1056300001000100010400FC000400000104190441
:1056400019FC000400040000000000000003000139
:105650000101190119FE0000000010041FFC0024C4
:10566000004001B4010C010400000000100410040B
:105670001FFC0004000400000000010401FC010400
:10568000010001FC0104010000FC010401FC008494
:1056900001000100010400FC0004000000F8010406
:1056A00001040104010400F80000010101FF00856C
:1056B00001040104008800700000000000700088F0
:1056C00001040104010501FF00010104010401FCC2
:1056D00000840104010001800000000000CC0124CE
:1056E00001240124012401980000000001000100B0
:1056F00007F80104010400000000010001F80004A3
:1057000000040004010801FC000401000180017094
:10571000000C001001600180010001F0010C00305C
:1057200001C00030010C01F0010000000104018CF7
:1057300000740170018C01040000010101810171FC
:10574000000E001801600180010000000184010CBE
:10575000013401440184010C00000000000000003D
:10576000000001003EFC400240020000000000007A
:105770000000FFFF000000000000000040024002A7
:105780003EFC0100000000000000000060008000FE
:1057900080004000400020002000000000000000C9
:1057A00000000000000000000000000000000000F9
:1057B00000000000000000000000000000000000E9
:1057C000000000000000000000000000000F803812
:1057D0000FFE380F803800000000000000000000BD
:1057E00000000000000000000100000600000C00A6
:1057F000003800003100000600000C0000380000F6
:105800003000000000000000000061800067F80721
:10581000F980006180006180006180006180006724
:10582000F807F9800061800000000000000000001F
:1058300001C0E003E0F00630080418081FFFFE0472
:105840000E080787F00381E000000000000001F06F
:1058500000060C00040408060C7001F9C0000E00DC
:10586000003BE000EC18070808040C180003E000F7
:1058700000000001E00007F003F818041C080417FA
:105880000807E1D003C0E00023B0003C0800200876
:105890000000100000000000000100003100003294
:1058A00000001C00000000000000000000000000DC
:1058B00000000000000000000000000000000000E8
:1058C000000000000000000000007F0001FFC00792
:1058D00080F00C00181000042000020000000000FE
:1058E000002000021000040C00180780F001FFC027
:1058F000007F000000000000000000000000000029
:105900000000000000004200006600006600003C4D
:105910000000180003FFC0001800003C00006600F3
:1059200000660000420000000000080000080000BF
:10593000080000080000080001FFC000080000087F
:10594000000008000008000008000000000000013E
:1059500000003100003200001C00000000000000C8
:105960000000000000000000000000000000000037
:1059700000000800000800000800000800000800FF
:1059800000080000080000080000080000080000EF
:105990000000000000000000000038000038000097
:1059A00038000000000000000000000000000000BF
:1059B00000000000000000000000000600001C00C5
:1059C0000070000180000E0000380000C0000700D9
:1059D000001C0000300000000000000000007F807C
:1059E00001FFE003807006001804000804000806A8
:1059F000001803807001FFE0007F800000000000BD
:105A00000000000001000801000801000803FFF881
:105A100007FFF80000080000080000080000000070
:105A2000000000000001C03802C0580400980401C2
:105A300018040218040418061C1803F81801E0F8EA
:105A400000000000000000000001C0E003C0F004FE
:105A5000000804080804080806180803F41801E7F9
:105A6000F00001E000000000000000000000030062
:105A7000000D00001100006100008108030108070B
:105A8000FFF80FFFF8000108000108000000000007
:105A9000000000E007FCD006080806100806100801
:105AA000061008061838060FF00607C000000000B0
:105AB0000000000000003F8001FFE0038430020886
:105AC00018041008041008041008071810030FF039
:105AD0000007C000000000000000000003C0000735
:105AE00000000600000600F80607F806180006E0A9
:105AF0000007000006000000000000000001E1E0D7
:105B000003F7F0063410041808041808040C0804FD
:105B10000C0806161803F3F001C1E00000000000B5
:105B20000000F80003FC30030638040208040208F1
:105B30000402080404100308F001FFC0007F000005
:105B40000000000000000000000000000000000055
:105B5000000070380070380070380000000000004D
:105B60000000000000000000000000000000000035
:105B7000000000000000301A00301C00000000008F
:105B80000000000000000000000000000000000015
:105B90000008000014000022000041000080800185
:105BA000004002002004001008000800000000006F
:105BB0000000210000210000210000210000210040
:105BC0000021000021000021000021000021000030
:105BD000000000000000000008000804001002009F
:105BE00020010040008080004100002200001400DD
:105BF00000080000000000000003C00004C0000412
:105C00000000080038080F380808380810000C3069
:105C10000007E00003C000000000000000003F801B
:105C200000FFE0038070020F1006708804C0880433
:105C30008308047F8802C09003012000FE4000001A
:105C4000080000180001F8003E0801C20007020029
:105C500007E20000FE00001FC80001F80000380045
:105C6000000804000807FFF807FFF8040808040804
:105C70000804080804080806180803F41801E7F0E7
:105C80000001E0000000000000003F8001FFE00391
:105C900080700200180400080400080400080400D2
:105CA000100600200780C000000004000807FFF86D
:105CB00007FFF804000804000804000804001802A4
:105CC000001003807001FFE0007F800000000400EE
:105CD0000807FFF807FFF804080804080804080884
:105CE000040808043E0804000806001801006000CB
:105CF000000004000807FFF807FFF804080804087C
:105D000000040800040800043E000600000600002D
:105D1000018000000000000000003F8001FFE00360
:105D20008070060018040008040208040208020338
:105D3000F00783F000020000020004000807FFF8EB
:105D400007FFF80408080008000008000008000029
:105D5000080004080807FFF807FFF804000800001F
:105D60000000000004000804000804000807FFF811
:105D700007FFF80400080400080400080000000001
:105D80000000000000000006000007000001040001
:105D90000104000104000307FFFE07FFFC040000EC
:105DA00004000004000004000807FFF807FFF804DF
:105DB0000C08001800003E0004C7800503C8060058
:105DC000F804003804001800000804000807FFF871
:105DD00007FFF804000800000800000800000800A1
:105DE0000008000008000018000060000000040027
:105DF0000807FFF807800807FC00007FC00003F8D1
:105E00000007C000780007800807FFF807FFF804C4
:105E1000000804000807FFF807000803C00000E0BE
:105E200000003800001E000007000001C00400F060
:105E300007FFF8040000000000007F8001FFE0037E
:105E4000807006001804000804000806001803000B
:105E50003001FFE0007F8000000004000807FFF829
:105E600007FFF80404080404000404000404000408
:105E70000400060C0003F80001F000000000000020
:105E800000007F8001FFE003807006008804008826
:105E90000400C806003C03003E01FFE6007F8400CA
:105EA000000004000807FFF807FFF80408080408CA
:105EB00000040C00040F00040BC00610F003F038BF
:105EC00001E00800000800000001E0F803F03006DF
:105ED0003010041808041808040C08040C08020602
:105EE000180207F00781E0000000018000060000B2
:105EF00004000004000004000807FFF807FFF8048E
:105F000000080400000400000600000180000400F6
:105F10000007FFE007FFF004001800000800000879
:105F200000000800000800000804001007FFE0045B
:105F3000000004000006000007E00007FE00041F48
:105F4000E00001F80000380001E0043E0007C00056
:105F500006000004000004000007E00007FFC00482
:105F60001FF80007C007F80007FF80043FF800078C
:105F7000C004F8000700000400000000000400084E
:105F800006001807C07805F1C8003E00001F800415
:105F900063E80780F8060018040008000000040009
:105FA0000006000007800007E008047C08001FF8D6
:105FB0000007F800180804E00807000006000004C5
:105FC00000000000000100080600380400F8040387
:105FD000E8040F08047C0805F00807C0080700184B
:105FE000040060000000000000000000000000004D
:105FF00000000000003FFFFE200002200002200001
:10600000022000022000020000000000000000004A
:1060100008000007000000C0000038000006000073
:1060200001C000003000000E000001000000000070
:1060300000000000200002200002200002200002D8
:106040002000023FFFFE00000000000000000000F2
:106050000000000000000000000000080000100028
:106060000030000020000030000010000008000098
:10607000000000000000000001000001000001001D
:10608000000100000100000100000100000100000B
:1060900001000001000001000001000000000000FC
:1060A0000000002000002000001000001000000090
:1060B00000000000000000000000000000000000E0
:1060C000000000F00019F8001B1800220800260844
:1060D000002408002410003FF8001FF8000008000A
:1060E000001800000004000007FFF80FFFF0001880
:1060F00018001008002008002008003018001FF0C9
:10610000000FC00000000000000007C0001FF000EA
:106110001830002008002008002008003C08001C5F
:10612000100000600000000000000000000007C038
:10613000001FF00038180020080020080020080484
:10614000101007FFF80FFFF0000010000000000023
:10615000000000000007C0001FF0001230002218ED
:10616000002208002208003208001E10000E200045
:10617000000000000000200000200800200801FFAF
:10618000F803FFF806200804200804200807200070
:1061900003000000000000000000000E000E6E0072
:1061A0001FF30031B10020B10020B1003191001F78
:1061B00013002E1E00200E00300000000004000816
:1061C00007FFF80FFFF80010080020000020000073
:1061D0002008003FF8001FF8000008000000000041
:1061E00000000000002008002008002008063FF8FA
:1061F000063FF8000008000008000008000000004A
:106200000000000000000000000003000003002068
:1062100001002001002003063FFE063FFC000000B5
:1062200000000000000000000004000807FFF80F55
:10623000FFF8000188000300002FC00038F800209C
:1062400038002008000008000000000000000000E6
:1062500004000804000804000807FFF80FFFF80016
:1062600000080000080000080000000000000020F6
:1062700008003FF8003FF8001008002000003FF839
:10628000003FF8001008002000003FF8003FF80031
:106290000008000000002008003FF8003FF8001050
:1062A00008001000002000002008003FF8001FF840
:1062B0000000080000000000000007C0000FF00010
:1062C00018300030080020080020080030080018AE
:1062D00030000FF00007C0000000000000002001A7
:1062E000003FFF003FFF00101100200900200800C0
:1062F0002008003038001FF0000FC0000000000030
:10630000000007C0001FF000381800200800200817
:10631000002009001011001FFF003FFF00000100D6
:106320000000002008002008002008003FF8003F7F
:10633000F8000808001008002008002000003000C5
:10634000003000000000000000000000000C780099
:106350001E180033080023080021080021880021AE
:10636000980030F0003860000000000000002000BD
:1063700000200000200000FFF003FFF800200800CC
:10638000200800200800003000000000000000008D
:1063900000002000003FF0007FF800001800000817
:1063A000000008002010003FF8007FF000001000FF
:1063B0000000000000002000003000003C00003F12
:1063C000800023F0000078000070002380003C0073
:1063D000003000002000002000003C00003FE000F2
:1063E00023F80000E0002700003E00003FE000210D
:1063F000F80001E0003E000020000000000020083E
:10640000002008003838003E680027800003C800DC
:106410002CF8003838002018002008000000000088
:1064200000002000003003003C01003F830023EC0B
:10643000000070002380003C0000200000200000CD
:106440000000000000000000003808002038002094
:10645000F80023E8002F88003E08003808002018C4
:1064600000007000000000000000000000000000BC
:1064700000000000000008000014001FF7FC3000BE
:1064800006200002000000000000000000000000E4
:10649000000000000000000000000000FFFFFF00FF
:1064A00000000000000000000000000000000000EC
:1064B000000000002000023000061FF7FC0014005E
:1064C00000080000000000000000000000000000C4
:1064D00000000000001800006000004000004000C4
:1064E000002000001000000800000400000400006C
:1064F0000C0000100000B5E70200020002007FF06F
:10650000421042107FF0421042107FF04200020819
:10651000020801F800000000D7D37FF000200040FF
:10652000008001000200FFF80200020002000200E9
:10653000020002000E0000000000BCBC1020102071
:10654000102013FEFC201020102015FC1884308829
:10655000D04810501020105051882606CAF501006E
:106560000120011001107FFC038005400540092037
:106570001110210841040102010001000100D2BAFA
:106580000080404027F8114001408278424816A818
:106590001AD02350222042204250028800000000DE
:1065A000BEA73FE020203FE020203FE00000FDF8B4
:1065B00085088508FDF885088508FDF88508000030
:1065C0000000B2E200084F8828880AA88AA84AA8D2
:1065D0000AA82AA82AA8422845088488888810384A
:1065E00000000000CAD44050204820400FF800406E
:1065F000E04027402240224022202A2833A82E189B
:10660000000800000000B3CC00001BF0E2102210D4
:1066100023F0F800200033F068806080A3F0208031
:10662000208027F800000000D0F2020001003FF8AF
:1066300020002FF02020224021803FF82088209049
:1066400040804080838000000000D1D5200010F8F9
:106650007E20444028F87E8848A850A864A848A80E
:1066600072A884501888610800000000C9AB1000AF
:1066700010003FE0404080807FF042104210421006
:106680007FF04000400840083FF800000000CCEEDA
:1066900020802FF8208027F0F41027F0241027F016
:1066A000241027F03410CFF802200410000000005E
:1066B000B3E404000200FFF80800104020207FF03F
:1066C000089008800880088010882088C078000022
:1066D0000000CEC4040002000200FFF81040104089
:1066E0000880088005000200050008803060C0189E
:1066F00000000000D7D604000200FFF880088008E0
:106700003FC0008001000200FFF80200020002000A
:106710000E0000000000CFD43FE0202020203FE00A
:10672000202020203FE008804890289028A0088062
:106730000880FFF800000000CABE00003FE0000033
:1067400000000000FFF80200124012202210420850
:10675000820802000E0000000000CDBC7FF8400857
:10676000440847C84848548843084CC87338408890
:106770004C08430840887FF800000000C6AC008049
:106780002080208020803FF02000200020003FC09B
:106790002040204020404040804000000000B4A540
:1067A00020403840484091F07D50555055507D5024
:1067B00055F054407C40545057F88C0800000000BD
:1067C000C3FE2220222027F8FA2027F0241027F0E9
:1067D0003410E7F020802FF821402220EC18000030
:1067E0000000CAE440804140F22044108BE8A00041
:1067F000F78824A827A834A8E7A824A8248825B8BF
:1068000000000000C8EB08000400040002000200C1
:10681000050005000880088010401040202040102E
:10682000800800000000C8AB0200020005000880DC
:1068300010402020DFD8020002001FC0020002002A
:106840000200FFF800000000B3CC00001BF0E210D3
:10685000221023F0F800200033F068806080A3F05D
:106860002080208027F800000000BCBC2080208011
:106870002080F7F02080208027E03220E220214095
:10688000208021402220EC1800000000CAF5020000
:10689000024002200200FFF807000A800A8012402E
:1068A0002220421082080200020000000000D6A749
:1068B00002000200FFF8020002007FE010201040FA
:1068C000088005000200050018C0E0380000000044
:1068D000B3D62080208023F0F880208027F828205D
:1068E0003020E7F82020222021202020E0E00000B6
:1068F0000000D7A8020002007FF004000400FFF8A7
:10690000080010003FE0002000401C8003000080D1
:1069100000000000D7A201004080200017F0008096
:1069200080804080008017F0108020802080408090
:106930004FF800000000C5FA204024402440F448ED
:106940002450276024403440E4402440244025481B
:106950002648E43800000000B7A2020022202210DE
:1069600044007FF8040008000FE014202440428017
:10697000810006C0383800000000B3C900A00090B4
:1069800000807FF8408040907C90449044A044A0D8
:10699000444858A84118820800000000B9A6010028
:1069A0000100F90023F021102110211021102110E5
:1069B0003910C21002100410086000000000D2C696
:1069C0000000002000780CE47904516810307E60EB
:1069D00019981A3C2FE448E40838003000600000A1
:1069E000D1A100000120012003FC622034200420FA
:1069F00003FC240021B021202220323E18000FE0A9
:106A00000000D4F10000000010FC1304110C3DF84C
:106A1000703E10D015907CF0503E18101BFE0230D6
:106A200000200000CFEE0000000003FE00607C406C
:106A300012FC11041106113611241F44794400C0C0
:106A4000009C01860000C4BF000000000FE03C185D
:106A5000200820043E04600460047E046004200CCE
:106A600020081FF001800000B6CC0000080011FCD7
:106A7000103E3EF82D8C2904490409043E8C50FC3C
:106A800010881EC811FC100E0000B0B400000040B9
:106A9000006012FE13023A427F4410C41BFE3C9871
:106AA0007190113011A00078004C0000C8B70000B0
:106AB000004000F878C41F8C313821EC2126413A7F
:106AC0007DE2272225FA3D26012401040000B6A814
:106AD0000000010001705FFC700420042FF8010029
:106AE0001100113821C431003F0063E0403800003C
:106AF000B3A4000000000818086008C00B001E00C6
:106B0000181C7FF01000118010E01838098E0F005B
:106B10000000B0B400000040006012FE13023A42D0
:106B20007F4410C41BFE3C987190113011A0007876
:106B3000004C0000B7B50000000007F80600240074
:106B400014F8078C04042408261825F0647C64C219
:106B500020801FC00000BBD8000000001FF03018CC
:106B60002008278C2C44284428442CC42784200443
:106B7000300C1FF803800000C7B60100210821086F
:106B80003FF800202220223EFF42229422103E1095
:106B9000221022283E2822440082CABD0048004418
:106BA00000440040FFFE004000403E4008400840D6
:106BB000082008220F12780A20060002BFAA00004F
:106BC0007FFC08200820082008200820FFFE08205D
:106BD0000820082008201020102020204020B7A2E4
:106BE00001001110110822003FFC0200040007F808
:106BF0000A080908111010A0204040A003181C0624
:106C0000CDF800007FFC40044004421452944A54E2
:106C1000442444244A544A54529461044004401485
:106C20004008D6D001000100010001003FF8210812
:106C300021082108210821083FF82108010001004E
:106C400001000100CEC4020001000100FFFE10108F
:106C50001010082008200440028001000280044037
:106C600008203018C006B2E2000427C414441454AB
:106C7000855445544554155415542554E554210460
:106C80002284224424140808CAD400282024102472
:106C9000102007FE0020F02017E011201110111025
:106CA000151019CA170A02060002000000000000B1
:106CB00000000000000000000000000000000000D4
:106CC000000000000000000000000000B4F300001D
:106CD000000000000018000010000010000010006C
:106CE00000100000100C3FFFFE0010000018000014
:106CF000180000340000340000220000620000414F
:106D00000000C1800080C001006006003808001C3F
:106D1000300000000000D4BD0000000000000300AF
:106D2000C00200B00200980260881F888C020FF039
:106D3000020C80022C887FDC88030C901B0CD01B7B
:106D40000C6013EE60131E64130CF413019C1B0201
:106D50000C27040421D800407FFC4007F800000005
:106D6000B4B400000000000003800803000C02E03F
:106D70000C06300C04198C08088C08008C18208C28
:106D80002FF08C48208C08208C08208C08208C0840
:106D9000608C09C10C08080C08080C08080C0C0CC5
:106DA0000C07FC78000010000000D0C200000000BA
:106DB000000002000801003C0133C03EC20008622E
:106DC00000044200048200049A0C3FFFFE010230DE
:106DD0000102300112301FE2300102300D42301941
:106DE0003630111430211430210830471030022081
:106DF00030000000D2BA00000000000000060018B9
:106E000003000C020C04FDF0011980011100423353
:106E1000083222F812421812651004E490056AB094
:106E2000056A200A71200861403860C01860C018E7
:106E3000616018623018641E087800000000BEA768
:106E400000000000000001004001FFC001004001FF
:106E5000004001FFC001004001004001FFC00100EF
:106E6000400000001064081FE7F8104608104608AC
:106E70001046081FC7F81046081046081046081F9D
:106E8000C7F8104608000000C6C10000000000005E
:106E90000800000FFFF80C00180C00180FFFF80C8A
:106EA00040900C30C00C10800C11100DFFF8083011
:106EB0008008308008308808309C1FFFE010208058
:106EC000102080206080204080408080030080006F
:106ED0000000B2E200000000000011000C09FE08F2
:106EE0000D860805864801A64841B64833B64813C2
:106EF000B64815B64805B64805B64805B64809A6C9
:106F00004809A64839A448182048185808184408C1
:106F1000188608190238060018000000CAD40000BC
:106F2000000000000001A01001D80800880C0088B3
:106F300004008400FFFE0000800000800400803C0C
:106F40000280047DC00408C00408400408400448CE
:106F500060048822050F3407381406E01C04000E74
:106F6000000006000000000000000000000000001B
:106F70000000000000000000000000000000000011
:106F80000000000000000000000000000000000001
:106F900000000000000000000000000000000000F1
:106FA00000000000000000000000000000000000E1
:106FB000D06F00080000002430000000D402000858
:106FC0000070000830000024B01E0000F00200082D
:106FD00018000000000000000090D0030090D003D3
:106FE0000000000000000000010000001000000090
:106FF000000000000100000018EF0000FFFF00008B
:040000050800029954
:00000001FF
